:10200000022024028DC4027533028DAC027988024D
:1020100034100234D032352D31322D3138000118D0
:102020001000AE0B7590FE758E04758F5290C20035
:10203000E030E203758FB075A8007581B275D000ED
:102040007580FF7590F675A0FF75B0FF75890075F6
:10205000980075880075B8007CFF90206579B1A75D
:102060008209A78332740A127428C22DC22C75F01B
:10207000087E04E5F0908000F090C3C0E065F05465
:10208000C07012E5F02440F5F0DEE890FB00E0209F
:10209000E448C38046908000E4F0908200E054DC85
:1020A000B41C139080007402F0908200E054DCB401
:1020B0005C04D22D80259080007440F0908200E076
:1020C00054DCB450159080007480F0908200E0548D
:1020D000DCB49006D22DD22C8001D350030256E7F7
:1020E000539003752DCC752E38302D03752E0812A4
:1020F0006AFEE52E908000F0752600126B1F752C8D
:1021000000126AD4532001C02EC02D792177000916
:10211000B97FFAD02DD02ED2119000E1E0540FC437
:10212000FB758901758C6A758A0075380A43896068
:10213000758DFF758BFF800075C83812654DD28C88
:10214000D28ED2CA75B83075A88A126ABE12659C42
:102150001267227401C0E0126B3BD0E004B411F5A9
:102160001289D145F0700E9000F47E03E030E00259
:10217000D235A3DEF79000147E04E4F0A3DEFC1257
:10218000745475F0001279FB05F030F2F875F00028
:102190001273E405F030F2F8128377E0539003B441
:1021A000EE02800F90345974EEF012839B128597E3
:1021B00012841D90001EE0A2E59218A2E1924175E2
:1021C000F08012864D1264B61264C675540875F01C
:1021D00081123373800112E527540FB40102800A83
:1021E000B4020280057432127428301417C214200D
:1021F0007F031289D17005E5F06009E48525F0744C
:1022000002126CD1E527547F4401B409028009E52C
:1022100027547F4410B4300574321274287549FF76
:102220008525F01273E4128E25753700C213754BA5
:1022300000753E00754600754700754800C21AC219
:1022400019C21DC279126B12754AAA30591675F05F
:10225000049000D8E0700DA3D5F0F9128E25207FF0
:10226000031289D1A2595002C259202B06202D03F6
:10227000022309302D24202C21C2D590C200E02059
:10228000E604D2D580145012C3E51A700DD2D5538E
:102290002DFB126AFE740A1274281270A565506034
:1022A0005974081274281270A5F5F06550604B300F
:1022B0002D11202C0E30E50B30D53F432D04126A32
:1022C000FEC2D585F0509000EAC0E0E054F0C3644F
:1022D000907001D3D0E0505330E01020F01975F029
:1022E00000C0E0126F20D0E030E10C30E13D20F181
:1022F0000675F001126F20022399302D0C202C0955
:1023000030D506432D04126AFE207803022399E596
:102310005AC4655A540FC0E0E55A540FC4535A0FBB
:10232000425A855AF0D0E07002806E753B00753CD1
:1023300000753D0020E50620E60330E72075F0003B
:10234000A2E792F3A2E692F530E50343F028E550C8
:10235000F4A2E52323540392E2F53D802A30E204FF
:102360007403800530E3027404F53CE5F0540FC4B7
:10237000423CE53C540F14F5F0207808740B1268C9
:102380004E30E11575F00412864D302D0C202C09CD
:10239000E5505460B46002C19330162220151DC36D
:1023A0001267B34017C2ACD2D3C2D4D2171238FCD2
:1023B000C21775A000C2D3759842D2ACC21630586D
:1023C00054C258C2D5302B4090C3C0302D039082E8
:1023D00000E020E5337402127428E020E52A126B35
:1023E00012E030E5FC302D08908000432E20E52ED1
:1023F000D2E5F074D2127428302D07532EDFE52E6B
:102400008003E054CFF0800D20D50A304607D2D5A6
:1024100090FB0080BC75F0009000D8E020E708A396
:1024200005F030F2F6A1EAC0E05403F05325FCE5D4
:10243000F054034225D0E0C0E0547CC36001D3D007
:10244000E0402212798930E10920E00302253F02B1
:1024500025B6C0F0E5F090008075F016A41268264D
:10246000D0F0022D2AC0E07432126CF4D0E0C0F03B
:10247000544FB4430302253D30E653C0E0740E12BE
:10248000684ED0E0B44907E0701F7410801EB44F4E
:1024900008A3E0701474158013B44A09A3A3E07074
:1024A00008741180077418800312681AC0E0E5F000
:1024B00090008075F016A4126826748AF0A3D0E00C
:1024C000F0D0F012798920E0030225B6A1D7B40A32
:1024D00003022552C0E0E5F090008075F016A412CA
:1024E0006826D0E0F5F0E05440448AF0A330E60CD2
:1024F000E582240FF582E5833400F583E0B4FF071D
:10250000E5F044F0F0803254F0B4F009E0C454F047
:1025100045F0F08024A3E0B4FF07E5F044F0F0803C
:102520001854F0B4F017E0C454F045F0F0D0F0C007
:10253000F0740712684E20E219D0F0A1EAD0F0E45E
:10254000126CF4128E2B1273E4E5F070EE754B00F2
:10255000A1EAD0F0C0F0E5F090008075F016A4126A
:102560006826D0F0E030E603022D2A12798920E0B7
:102570006630790DA3A3E0B4EE02803A74021268CB
:102580003CC0F0A3E0F5F074FFF0A3E0C0E074FFFE
:10259000F0E582240EF582E5833400F583E5F0F062
:1025A000A3D0E0F0D0F0E582C39411F582E58394E6
:1025B00000F583022D2AE5F0C0F090008075F0163A
:1025C000A4126826E044CAF0D0F07472126CF412BF
:1025D0008E2B75F030800874F2126CF475F03C307C
:1025E000790630260312A6278000301003022683C6
:1025F000307B04E4129D77307C03129B9030196984
:1026000075F0FF3007087414D5E0FDD5F0F5903271
:1026100093E012681AF5F0A3E012681A900082F0B5
:10262000E5F0900081F0903295E0F5F0A3E07004C1
:10263000E5F0600BE0900091F0E5F0900090F090F4
:102640003292E020E20975F000900080022D2AC24B
:10265000A8C2AA9032987877E0F6A308B87BF9531D
:1026600021FC7D221291F380DD2010173078143088
:102670005F0312A1D5201C0B200508307D05C27D0B
:1026800012A209126AEF30E02D7EC8126AEF30E024
:1026900025DEF8753B0075F04012864D202C113078
:1026A0002D0E74FF127428432D04532DF7126AFE69
:1026B0004387020226B3305A08C25A75F0411233DA
:1026C00073E5547034755408302D18908000432EF3
:1026D00020E52ED2E5F074D2127428532EDFE52EB9
:1026E000F0801690C3C0E526F4540FD2E5F074D202
:1026F000127428E526F4540FF0753B00E53BB41046
:1027000003022B98302D06B40403022B9804F53BEA
:10271000901E9A75F008A4126826C082C083A3E0B8
:10272000D083D082A2E7921EF5F0E53B1271CFF57F
:102730003C65F05403700AE5F00303653C54036004
:10274000BBC0F0742875F0FAD5F0FDD5E0F7D0F0F5
:10275000E53B1271CFF53C65F05403701A921E9060
:102760001E9BE53B75F008A4126826E003035403A2
:10277000653C6088022A98301E10E53C30E10BF47D
:102780005407F5F012864D022A80921E75F00074EF
:102790001412684E54E07015A3E0540FB53B0E3090
:1027A0001E06E4126D33800A126DBC800505F03000
:1027B000F2DD5325FC8525F0740212684E543FB5B6
:1027C0003B03022829A3E0541FB53B030229A07450
:1027D0001412684E54E0A3B48012E0541FB53B0CB1
:1027E0009000DE302901A3E06002800FE52554034C
:1027F000B40303022A2305250227B52323F5F0306D
:102800001E18740212684E541F1271CF5004052511
:1028100080A3B2F0757000126F20B2F0E412684E1F
:1028200075F000124EE7022A80E525540375F01674
:10283000A4900080126826E0601120E73B301E382B
:102840007401F0307803437180802D8525F0302DA0
:1028500004B2F0800520F120B2F1740212684E300B
:10286000E716543FB53B11E5F0540375F016A490FC
:102870000080126826E070C28525F0740012684E50
:10288000543FC0E023901F212582F582E583340068
:10289000F583E054816481301E077005D0E0022783
:1028A0005F301E06E020E711600F8525F0741412DA
:1028B000684E54E0301E387003022934740B1268DD
:1028C0004EA2E59000DE302901A3E07067E5250304
:1028D0000354C0D2E54002441EF0202909D265D23B
:1028E00066126AD4804ED231D233126B1F8045F506
:1028F000F0A3E0541F42F09000DE302901A3E02352
:102900002365255403601C30F709E5F0541F12714C
:10291000CF4021E4F0532C0F126AD45326F0126BEF
:102920001F801130F60EE0600B8525F0B2F0757057
:1029300000126F20901E9CE53B75F008A4126826DB
:10294000E0201E07C0E0C39195D0E020E702700DA3
:10295000201E19E4F0D0E0127043022A6BD0E02070
:102960001E07E4F0127043418002275F8525F07452
:102970000212684E20E609D0E0126C154004416B4B
:10298000D0E0C0E08525F0740B12684EA2E5D0E0DF
:10299000400675F000124EE78525F0126E21418049
:1029A000901E9AE53B75F008A4126826E0547FF566
:1029B000707006201E11022A80201E03022A231294
:1029C0007BF6400302275F74158525F012684E548C
:1029D0000F600512706E4038E52554032323902FB5
:1029E000A82582F582E5833400F583E020E32120E9
:1029F000E2218525F0E412684E543F23901F2125E3
:102A000082F582E5833400F583E030E70620E103B8
:102A100002275FE570757000C0E0126F1DD0E07096
:102A200002805D901E9CE53B75F008A4126826E0CC
:102A3000547F7001F0C0E0A3E0201E1830E607D0FC
:102A4000E060280226FCD0E06021740112683C742A
:102A500000F0802CD0E070B8E06010543F2304C038
:102A6000E0740112683CD0E0F08015301E08127C42
:102A70001D409DD3919575F000A21E92F012864DD7
:102A8000901E9BE53B75F008A4126826E054FC53A9
:102A90003C03453CF002275FA3E060030226FC757F
:102AA000F000753A01901FA4E0C2F054E06005B454
:102AB000203AD2F0E0541FB41F35C0F0C03CC083B0
:102AC000C082A3A3E0D2D56016C2D5F53CE53B9009
:102AD0001EA075F008A4126826E0B53C02D2D5D03D
:102AE00082D083D03CD0F030D5758006022B5FB504
:102AF0003B6DA3E0C40354076003B4010AA21E3077
:102B0000E001B392D58010B40704D2D580095403F4
:102B1000C2D5B53C02D2D5E582240420F0022406B9
:102B2000F582E5833400F58330D521E0B4FF14C08D
:102B300083C082C0F0E53B127C1DD0F0D082D083F0
:102B4000B38003127BF64004D2F780031272E9745B
:102B50000130F00D74031274287407800441A874C6
:102B60000C2582F582E5833400F583053AE53A7059
:102B7000EC901E9BE53BC0F075F008A4126826E5BA
:102B80003C2323540CF5F0E054F345F0F0D0F03042
:102B9000F603022C880226FC900080E0B40106C2F5
:102BA00028C2298027900096E0B40106D228C229C5
:102BB000801A9000ACE0B40106C228D229800D90A2
:102BC00000C2E0B40166D228D22980008525F0E455
:102BD000126CF4A3E0F543A3E0F544A3E0547FF5C1
:102BE00045A3A3A3E0F54BA3E0F53EA3E0A2E19249
:102BF0001A75700053718042715404F537D21385F1
:102C000025F0E57120E012E582240AF582E583349F
:102C100000F583E0D2D5B4FF05C2D51273E4127972
:102C200089F52920D5030230F3022E53753B01E5C7
:102C30003B901E9C75F008A4126826E0547FB401F6
:102C400047E0C2E0F020E722A3E020E607E53B12E0
:102C500071CF5034127C1DA34015E05403F53CA302
:102C6000E0D2E7F075F01112864DD391958012E015
:102C7000540FF53CE0B2E0F0E53C0303653C30E086
:102C800007D21E75F04041A2053BE53BB41103029B
:102C90002245022C2FC083C08292F7E53BC0F0751D
:102CA000F008901E9EA4126826D0F0E0600DA2F7F6
:102CB00014F5F092F7D2F6E4F0800353F08074023A
:102CC00012684E543FB53B50740712684E30E148CD
:102CD00020E403E4800274FFA2F120F008F535C27D
:102CE0005B925D8006F536C25C925E30F705126C31
:102CF0003F8003126CBCB4FF00B3E5F05403C0F096
:102D000030F70A75F015500875F00F800375F01450
:102D1000127961D0F020F60D05F0202D0530F29EDD
:102D2000800330F199D082D08322C205C20453259A
:102D3000FCE5F054034225128E2B754A00740A12EA
:102D400068317806E0700BA3D8FA75310575320545
:102D5000803A9000DCE0B4AA02801A7543037544FF
:102D6000D9754500757100C21AC2137537A0740475
:102D7000126CD1E13E8525F0741412684E54E07057
:102D800019A3E0541F601312706E500E7460126D20
:102D90003353900375A0000221D7126ABE1279FB4B
:102DA000301810304D0D7448126CF47404126CD14C
:102DB0000221D7754B00E525540375F016A4900049
:102DC00081126826E0B4FF02801054F0B4F005E0F0
:102DD000540F8001E0126803F54BA3E0B4FF0280BA
:102DE0001054F0B4F005E0540F8001E0126803F5D0
:102DF0003E8525F0E54B7007740D12684EF54BC209
:102E00001AB414004007B41E005002D21A300C024B
:102E1000C2AC127DA9D2AC303407C234C2137537AC
:102E200001E53720E02D5371FE8525F0740B126803
:102E30004E30E61FE525540375F016A4900083126A
:102E40006826E0540CB40C0BE054F04403F537C290
:102E5000138039E525540375F016A490009212688A
:102E600026E0B4FF0280030231B1201319E5375484
:102E7000FBB41018E57320E60B8525F0740B12687F
:102E80004E30E408D213201A06022F44022F3EE5EA
:102E900072A2E3035401F5F092F1E54BC2E0B414E1
:102EA000028011B41602800EB41802801EB41A02F9
:102EB0008026807C801730F114E54BA2E0B392D5D8
:102EC000E53EF53A60071272E9804780007537FAEF
:102ED000753EFAC213022F3E30F1F2E54BA2E0E557
:102EE0003E402212A003501D0221D740188525F034
:102EF000740F12684EF5F0A3E06009B53E06D37575
:102F00003A828009C375F0FE753A00E53E92E712F9
:102F10008BC82019168525F07405126CF420F00575
:102F20007535058003753605126C3FD21302326C7D
:102F3000E54B20E004E53E809430F19180D4126DA1
:102F4000D902326C2019FA8525F0741412684E5497
:102F5000E060209000DE302901A3E06003022FF63C
:102F60008525F0B2F0E412684E543F126C15500300
:102F7000022FF68525F0740F12684EF5F0A3E0607D
:102F800057C0E0C0F0127C69501BE57230E309D3F2
:102F9000D0F0D0E04042805EE5F0B4C00040F1B433
:102FA000FC00B380EB8525F07460126D337403125E
:102FB0006CD1E572A2E350D8D0E0B4010274FCD029
:102FC000F06015C5F0F53E4480C03A753A02128BA8
:102FD000C8D03A754B7FD21A8525F0E412684E545A
:102FE0003F23901F212582F582E5833400F583E09D
:102FF00030E70820E005437101E13E740B12684E92
:1030000030E34A53707FE57060EC901F9875F00CC8
:10301000A4126826E054E0B48033E0A3A3A3A3A3E2
:10302000A3A330E00F8525F053F00305F003D5F09E
:10303000FC30E00CE06016D2D5F53A1272E9800D52
:10304000A3E060B2D2D5F53A1272E980A9304B14F0
:10305000E572A2E7500320E30BE53792E7C2E6F5FD
:1030600037023149126F1D2057030230F3307909BE
:1030700030260675F00E12A6278525F0740C12680E
:103080004E543F127BCEE5824004940380029406A6
:10309000F582E5839400F583E0543FB43D0050028F
:1030A00024025372F7C0E0E525540375F016A4908E
:1030B0000080126826D0E07002740AF08525F07452
:1030C00072126CF4A3E543F0A3E544F0A3E054804E
:1030D0004545F0A3A3A3E54BF0A3E53EF0A3E537F8
:1030E0005404A21A92E1F020F004C2A88002C2AAFD
:1030F0000222455390038525F0740B12684E30E38D
:1031000002416CE57220E106E57060F5802FC04356
:10311000C044C04512428FD045D044D0434025859D
:10312000F090E0540FB4011CA3E0539003127BF61F
:1031300085F090E582255BF582E0539003D2D5F5CA
:103140003A1272E9539003416C8525F01273E4E55D
:1031500025540375F016A4900080126826748AF036
:10316000E5822404F582E5833400F583E020E7035B
:10317000A38009E545D2E7F0A3E570F0E582240DD0
:10318000F582E5833400F583E54BF0A3E537F0A342
:10319000E543F0A3E544F074728525F0126CF43039
:1031A000790930260675F03C12A627128E2B0222D2
:1031B00045F5F0A3E020E60385F04BF5F0A3854547
:1031C00048854447854346E0F543A3E0F544741140
:1031D00012683CE0547FF545B54822E544B5471DEB
:1031E000E543B5461830F611754B635372F7126F0D
:1031F0001D753700D21302326CC0F0803330F60CEC
:10320000854845854744854643022E6AE53753374E
:10321000FBA2E272F292F254FBB41007E57330E6BF
:1032200002D213A2F7C2F7C0F0E572500820E305FE
:10323000C213433780201305126DD98028E030E790
:1032400024C2E7F0A3E0C0E0126F1DD0E06007F5F4
:103250003AD2D51272E930570C85484585474485E6
:10326000464302306DD0F01288F580031287422069
:103270001909307912E5255403F515129E6B307942
:103280000675F08012A62730132CC0D0C0E0E5717F
:1032900020E01FD2D5128CC3E5487008E5477004C2
:1032A000E546600E854845854744854643C2D512AC
:1032B0008CC3D0E0D0D05031C0E0B40304D234800D
:1032C00005B40425D21875F0217173D0E08525F07E
:1032D00030E009744C126CF4740780077448126C67
:1032E000F47404126CD10221D7301349301A46E528
:1032F0004BB47F0E8525F0740F12684EF5F07443C1
:10330000801654FCB4182E854BF020F003433E8009
:10331000744330F12075F0FE900203F0A37480F046
:10332000A3E53E533E7FF0A3E5F0F0740A12742843
:103330007404125F0A75F000717330131D20191A9E
:10334000201A17E5487013E547700FE546700BE546
:103350007230E3064337400231498525F053F003CC
:10336000E5F09000D82582F582E030E703022427BB
:103370000221D7753A01901FA4E0753B0C54E02060
:10338000F005B440758017B46070A3153BE04401AC
:10339000B5F067A3A3A3153B153B153B804EE05446
:1033A00007600714652554037050E0A3153B30E413
:1033B0000A301346E57120E0418008301305E571BD
:1033C00030E037E0B4FF0280045537602DA3153B91
:1033D000E0B4FF028003B54B21A3153BE0A3153BEE
:1033E000B4FF028007B54412E0B5430EA3153BE0DD
:1033F000127BF65005D2D51272E9E53B2582F582A3
:10340000E5833400F583053AE53A70012202337909
:109B9000C0D0C2D3D2D4C27C207E03029C0A9002E1
:109BA000057412F0C03A902D27753ABFE0F5F0A386
:109BB000A3E030E749A2E392D5C2E3A2E2F0E5F0E8
:109BC000C082C083129C60900207F05017600FB4EF
:109BD000C00730D50F741E8005B480084401A3F07F
:109BE000744280027402900206F0900201E53AF09D
:109BF0007406D3C0F0125F3DD0F0D083D082A3A30F
:109C0000A3053AE53AB4CFA4D03A202603D0D02217
:109C1000902D77C0255325FCC082C083E030E22719
:109C2000A2E392D5C2E3F074108525F012684E606D
:109C300016129C606003B4C00575F0148006B480F1
:109C40000675F00F12A627D083D0827408126831EF
:109C5000E5255403B40305D025D0D022052580B8CE
:109C6000C0D0C0F06019127C695017E5F06010D2C6
:109C7000E0B4FF02800954C0B4C00B74808009E4D2
:109C8000800674C080027440D0F0D0D022C0D0C210
:109C9000D3D2D4C0E09002057412F0A37440F0A3B4
:109CA000E4F0A3740F500274B3F0900201D0E0F01E
:109CB0007406D3125F3D22C0D0C2D3D2D4C0A8C292
:109CC000AFC082C083EDB40400500512679E403ED1
:109CD000207E09D083D082D0A8D0D022900201ED7E
:109CE00024BFF09002058583A0A882EB54C0B4C0C5
:109CF00054D083D082E0B41C027F02B41E027F12D3
:109D00008FF0E0F2A308DFFAE5F024028056D226B5
:109D1000D27A74562DF8E6F5F0900200700474A023
:109D2000800274A1F0A3A37410F0A3EDF0A38583C7
:109D3000A0A882EB0303035403F208EB5407F208D4
:109D4000EEF20880077413F208EBF208D083D08299
:109D500020D5057F0012A183EF2404307A06240564
:109D6000900201F0D0A8D3125F3DD0D022C0D0D253
:109D7000D5C2D3D2D48010C0D0C2D5C2D3D2D4C21F
:109D80007B207E03029E21C0E06003C394BF902D20
:109D90002975F005A4126826D0E0C03A600575F078
:109DA00001800574BF75F010F53AC0A8C2AFC0833A
:109DB000C082900205741630D502741FF0A385830B
:109DC000A0A882D082D08312A1B1D0A8E030E7430E
:109DD0005403FF740212683CE0129C60A3A3C0828B
:109DE000C08390020BF030D511A3E528A2E492E1E4
:109DF000A2E592E05403F0A3EFF0900201E53AF0FF
:109E0000740930D502740BD3C0F0125F3DD0F0D08E
:109E100083D082A3A3A3A3A3053AD5F0AFD03AD2AF
:109E2000D5202603D0D02230D505740A127428C05C
:109E3000A8C2AFD27A90020074A0F0A3A37410F06D
:109E4000A374FFF0A37404F0A3E4F0A3E51F126869
:109E500003F0A3781D7F04E6126803F018A3DFF770
:109E6000E502126803F07F0A029D58C0D0C2D3D227
:109E7000D4C0A8C2AF7F00301908E552C394BFFD1B
:109E8000800BED12679E4005D0A8D0D0229002072B
:109E90002013167B5020190474037E0490AAB1C2CB
:109EA000D5129CB7D0A8D0D0228583A0A882301923
:109EB0000FE54BC2E0B41C047B0080027B80800471
:109EC0007B037E04301A03029F7CC016C071C072EF
:109ED000C010757B00757C00757D0085447E8543D0
:109EE0007F1299A5D01090AC4912A183E57144303E
:109EF000F208E57212A171E57312A1717F022019B7
:109F0000027F0A7420F208DFFC7F102019027F18FC
:109F1000D072D071E54B800CC0D0C0A8C2AFC016C3
:109F2000C2D3D2D4F5F0D2F7902D977E1FE0B5F0D2
:109F300002802C7411126831DEF3C2F7E5F070056F
:109F400090A7958006B4010890A7C712A18380202E
:109F500090A7F112A183E5F012A16E0F0F8011A35B
:109F60007E10E0600BF208B8000205A0A30FDEF23D
:109F7000D016D2D5129CB7D0A8D0D022E54B12680B
:109F80001A30E33520E00D90AAB18000C082C08372
:109F9000E53E8049E53E127C6930E70590AB3980AB
:109FA0000890A9A1500390AA29C082C08390A8213B
:109FB000E53E700390A85D802430E20E90A9193030
:109FC000E00390A95D30E1BF80DF30E10E90AAF59B
:109FD000C082C08390A8A1E53E800280AAC0E012A2
:109FE000A183D0E0600512A16E0F0F20190B75F050
:109FF000087420F2080FD5F0FAD083D08212A18322
:10A00000029F72C082C08320190FE5255403126796
:10A010009E4006D083D082C322C0F0C0D0C2D3D22B
:10A02000D4C03B753B01901E9AE53B75F008A41225
:10A030006826E0B47F0280207406126831E0601860
:10A04000B53E028004E53E700FE53B1271CF50082B
:10A0500012A078500302A062E53B04F53BB411C6A0
:10A060008007D330F40312A627D03B92E0D0D0A2D1
:10A07000E0D0F0D083D08222C0D0C082C083C2D3CF
:10A08000D2D42007FD7F009002078583A0A88230EC
:10A09000190AE552C394BFFD7B608009E52554038E
:10A0A000FD7B037E0490AB7D12A183E8C3940EF880
:10A0B000E53B12A16EE8240CF8ED20191475F008A8
:10A0C0007420F2080FD5F0FAED75F008902D778026
:10A0D0000675F005902D29A4126826E030E406D319
:10A0E00090AC058004C390ABC112A183D2D5129C61
:10A0F000B77496127428500575F0148004740080AB
:10A10000047480D219D083D082D0D0A2E722C03A82
:10A11000C03B753B01901E9AE53B75F008A41268A0
:10A1200026E0B47F0280297406126831E020D50C45
:10A13000B53E028014A3E0B53E16800DC03BF53B52
:10A14000E53E127CA5D03B4007E53B1271CF800174
:10A15000C3E53A13F53A053BE53BB40904C03A8040
:10A16000B4B411B1853AF0D0E0D03BD03A221268B5
:10A170001AC0E0C4540F4430F208D0E0540F443009
:10A18000F20822C0D0C0F0E528C45403F5F0E5F091
:10A19000600AE493A3B42FFA15F080F2E493B42F8D
:10A1A00005D0F0D0D022F208B8000205A0A30F809D
:10A1B000EBE51B126803F208E51A126803F208E5E2
:10A1C0001C126803F208E51D126803F208E51F126D
:10A1D0006803F20822C25FC2ADC0D0C2D3D2D47F1E
:10A1E0000790020074A0F0A3EFF0A37413F0A3741F
:10A1F000FFF0A3E4A21CB392E0F0D3D27AEF125F97
:10A200003D7410127428D0D022C2ADC0D0C2D3D2B7
:10A21000D402A60C900308ED75F00CA4126826E099
:10A2200030E6EE30E10302A2D4C226A3A3E0F5F0AB
:10A23000E55614B5157BC0F07F029002007402F061
:10A24000A3E5F012A76A7400F0A3E557701174013A
:10A2500062F0F00FA3745662F0F00FA302A297749D
:10A260000762F0F00FA3745562F0F00FA37401625F
:10A27000F0F00FA3E557B4FF0B7E0462F0F00FA3DC
:10A28000DEF9800FE47E03F00FA3DEFBE55762F0FA
:10A29000F00FA3E4F00FA3E5F012A76A7403F0D364
:10A2A000D27A0FEF125F3DD0F04006755600755719
:10A2B000007F049002007402F0A3E5F012A76A7414
:10A2C00000F0A37400F0A3E5F012A76A7403F08015
:10A2D0002402A60CD22674562DF8E6F5F07F0690DF
:10A2E0000200700474A0800274A1F0A3EFF0A374C4
:10A2F00011F0A3EDF0D3D27AEF125F3D500E30266D
:10A30000D074562DF8760012A1D580C530260302F0
:10A31000A4AC90022A12A78B70B712A78BFE12A7CB
:10A320008B60AE12A78BB4410302A34AB44203026E
:10A33000A36AB4430302A390B4AF0302A3E6B42814
:10A340000302A3FBB4618A02A3FE12A78B787A12E0
:10A35000A78BF618B876F87505225321FCED540347
:10A3600042211291F3D27902A6177F0B12A78BDF3D
:10A37000FB12A78B603AB4060040027406FF232349
:10A38000232402F505787712A78BF608DFF980CA37
:10A390007F0D12A78BDFFB12A78BB40703D38001BD
:10A3A000C3C0D012A78B12A78B12A78B7004D0D07A
:10A3B0008049B4080040027408F5F01423232324D4
:10A3C00001D0D0C0D040022401F50512A78B25058D
:10A3D000F505787712A78BF608D5F0F8D0D05003A2
:10A3E00053777F02A35A12A78B20E00620E10702D1
:10A3F000A60CE402A4DC740102A4DC02A60C7F0615
:10A4000012A78BDFFB12A78BC03BA2E0B392D5C291
:10A41000E0B41203048009B414028004B4161914C1
:10A42000F53BED75F003A4253B126803F53B75F091
:10A4300000A2D592F012864DD03B02A60CC0D0E50A
:10A44000F0B4AF419002007F14E4F0A3DFFC90026F
:10A450000074A0F0A37414F0A3740DF0A3EDF0A3A6
:10A46000740CF09002087432F0A3A37403F090020D
:10A470000E7F0474FFF0A3DFFC7F14D3D27AEF12B7
:10A480005F3DD0D022900200E5F0F0A37407F0A366
:10A490007412F0A3EDF0A3E4F074562DF8E6F5F095
:10A4A0007F07D3D27AEF125F3D1264C6BD030574F5
:10A4B0000712742890022AC2D5E0FFA3E0A3B411CA
:10A4C00005BF07118015B40B03A38056B40C03A37A
:10A4D0008050B40A4AE0A36049801AE013B3E44014
:10A4E00001F48DF005F033D5F0FC4004425A8002AF
:10A4F000525A02A60CB41A077577007878800FB408
:10A5000020077505227877800CB422137877E05401
:10A5100001F0750529E0F608A3B87CF902A35A02F8
:10A52000A60AE0A3FF74081274288583A0A882BF3E
:10A530000146ED540375F008A4902D78126826E2C8
:10A540007F0375F00CB5F028E0602B7F02E0B4FFCC
:10A550000474EE800312681AC0E0C4540FF208D0ED
:10A56000E0540FF208A3DFE5181818187F048008DC
:10A5700005F0A3A3DFCF7F01C0A8C2AFED540375E0
:10A58000F016A4BF05004005D0A802A60C900080DC
:10A59000126826E05440448AF0A3C3C01730E60D89
:10A5A000E582240FF582E5833400F583D3E2F0DF02
:10A5B00002800CC4F5F008E245F0F0A308DFEED00D
:10A5C000E0402E03540312683CE0FFED540375F0A5
:10A5D0000CA4900308126826E030E215EF1268031D
:10A5E0009002078583A0A8827F007B037E0A129FCA
:10A5F00018D0A8ED54039000D82582F582E5833465
:10A6000000F583748AF0D279800D7600201C080D45
:10A61000BD040040057DFFD0D022740230260274B4
:10A620000512742802A214C2ADC0D0C082C083C279
:10A63000D3D2D420264AED90030A75F00CA41268F8
:10A6400026E0F5F09002007F047402F0A3E5F0121A
:10A65000A76A7400F0A3740262F012A76A744862D9
:10A66000F0F0A3E571A2E07402301304400274011B
:10A6700062F012A76AE5F012A76A7403F002A7500D
:10A68000740A1274289002007F14E4F0A3DFFC9097
:10A69000030AEDC0F075F00CA4126826D0F0E0704B
:10A6A0000474A0800274A1900200F0A37414F0A3BB
:10A6B000740DF0A3E5255403FDF0A3E5F030E71495
:10A6C00030130FE57120E00AA2E7742250067420CF
:10A6D00080027408F020F006A37432F0801620F196
:10A6E00007D2E1C2E0C2E4F0A374DCF0A37405F089
:10A6F000A37405F090020820F2057432F0800B7408
:10A70000DCF0A37405F0A37405F090020B20F405AF
:10A710007432F0800B74DCF0A37405F0A37405F0C0
:10A7200074562DF8E6F5F090030AEDC0F075F00CC4
:10A73000A4126826D0F0E0B4FF02E58AF61263BFE7
:10A7400090020E7F047883E6F4F0A318DFF97F14FB
:10A75000D3D27AEF125F3D3026095007D083D082E2
:10A7600002A444D083D082D0D0220FB40202800D44
:10A77000B403028008B41B028003F0A3220FC0E0E0
:10A78000741BF0A3D0E0D2E7F0A322E0B41B04A333
:05A79000E0C2E7A32276
:10341000C236C2A9C0E0C0F0C0D0C083C082C0A084
:1034200075A001C215C2D4D2D3C090539003309975
:103430000B209C030234B71264B68063E599C298EE
:1034400020052F200416F5F0902022E493B5F04FCC
:10345000D204C20578007D007EFF8043B45F04D2B1
:10346000218003B53906D205C2048033C204C205E7
:10347000802DBE0008B4041CC2AC02363ABD000C5C
:10348000FD0404FE90007AE0F53080136530B8004A
:1034900006B4FF0302378875A001F2081E800053AE
:1034A0009003D0E054FD4290D0A0D082D083D0D001
:1034B000D0F0D0E0D2A932C299126583BD000302D8
:1034C0003788BD010474048002E2081DF59980CF9D
:1034D00053C83F755305C237C2A9C0E0C0F0C0D081
:1034E000C083C082C0A075A002D215C2D3D2D47549
:1034F000F0007400C2D5126448C09053900320F7C6
:103500000C30F60302361F1264C602349FF5F03009
:103510007821C0107829E2D010C2E0B4A002800166
:10352000D3E5F030070540420235BB30060B4022A0
:103530000235B1200734200619902022E493B5F01B
:1035400057D206C2077829E4F278007D007EFF0298
:103550003609B45F04D2228003B53907D207C20608
:10356000023609C206C207023609BE0008B4041DAD
:10357000C2AC02363ABD000DFD0404FE90007AE0B4
:10358000F53002349F6530B80006B4FF0302378E71
:1035900075A002F2081E8071E5F0C2E0B4A06A30A6
:1035A0007867302664E5F0D206C2077EFF7829806E
:1035B0000AD20714FE700302378E0475A002B83DCC
:1035C0000050F4F2081EBE00CD201C02D25F782904
:1035D000E2F5F008E2FF28C39404F8E230F0026458
:1035E000025403FD1264C690022974562DF8E62099
:1035F000F007E4F675F0A0800375F0A1C2D5126360
:1036000060600375F0AF12A43D20911075F0007456
:1036100000C2D512644830F70302350D02349FBD55
:10362000000302378EBD010474048002E2081D7598
:10363000F082D2D512644802349FA215923E90F3D4
:10364000FCE58F30E10390F9FF8000A3E58370FB78
:103650008DF07C007D00902022E49312640BE5390C
:10366000203E053021078003302202745F12640B74
:10367000E5F012640BC0F07800E2653012640B08CC
:10368000D5F0F6E530600E75F00490007AE0126433
:103690000BA3D5F0F8E265308DF0B5F00E08E265C9
:1036A000308CF0B5F005D0F0023748D0F0E530604E
:1036B0002B1263E0400B1236E140217530000237D7
:1036C0004890001EE0C2E7F01236E150F190007A17
:1036D0007400F075300075F0E3024372C21B0237CC
:1036E000857800E26530B471028017B478028012E8
:1036F000B45602800DB457028008B477032011023B
:10370000D3227C007D007800902022E49312640B89
:10371000E539203E053021078003302202745F1214
:10372000640BE5F012640BC0F0E26530F212640B3A
:1037300008D5F0F5D0F0E26530B50D0A08E2653045
:10374000B50C03C38001D3229000E1E0540FC4F50F
:1037500003203E0A755408302102D21B8007C203A1
:10376000302202D21BADF01D203E0575A001800362
:1037700075A0027800E2F5F0F9903796E4A3A3A3D0
:10378000A393B42F0F203E061264B602349F126436
:10379000C602349FB5F0E5740173010238F181026D
:1037A00038F1C10238F102023C8103023DF3050207
:1037B0003F6006023F94070242EC0802436A090296
:1037C00043A70A0244B80B0244BB0C0245EA0D02AF
:1037D000464A0E0246AC100246E71102483B12026E
:1037E00042F6130248941402489715023F4A160203
:1037F00048EC170243022002492121024AAF22026B
:103800004B192302491B25024B6126024BC431028E
:103810004D6F32024DD333024E8834024EA2350230
:103820004FBF37024FD83802501A4002475F41025B
:103830003C4F43025033440251364502513946024F
:103840003F8E4B025193510252EC5402532B5502BE
:10385000535E5602539C570253EA7002543D710264
:10386000548A720254EA73025631740256CD7502BC
:10387000571476025763770257D57802582F79028A
:1038800058C77A02598A7B0259987F025B692FC216
:10389000115390038DF0C0F07C007D007800E2C0F1
:1038A000E0E8B40300D0E040036530F212640B0896
:1038B000D5F0EBE530600E75F00490007AE012640C
:1038C0000BA3D5F0F8EDF208ECF2D0F0ADF07800F3
:1038D0000D0D0D301702C322201508759842D2AC89
:1038E00002349FE2081D75F082D2D512644802347A
:1038F0009FC217C211C202B90147805275A0019040
:1039000000E1E020E717900004E0B4011279019093
:1039100034591283B3903459D20F0239F6C20F785A
:10392000007441F208E539F2087405F2087471F286
:10393000089000EE7D04E0F208A3DDFA7D0802386D
:103940008F7400A20192E66920E6030239CEB2012B
:10395000128391E0B4EE24C082C0831283C5D08369
:10396000D082502312845F40147012539003900051
:103970001EE030E4129034591283BC805E128391B1
:1039800074FFF07901806F12844B5028C218C23442
:10399000539003900004E4F090001EE054C7F090B0
:1039A000345912839B1285979034591283B3903403
:1039B000591283BC78007441F208E539F2087401A9
:1039C000F2087460A20192E4F27D0402388F12833F
:1039D000911283BC128396A955801B300F04B2014B
:1039E00080EC1283961283B312839612844B4004A8
:1039F00079018002790A755500C090C083C0825356
:103A0000900378007441F208E539F2080830160B8B
:103A10009000EE7E04E0F208A3DEFA7460A2019248
:103A2000E4F208D082D083D09012845F402C6005ED
:103A30001284C58025C082C083C09053900390003B
:103A40001EE0A2E4C2E4F0D090D083D0824005749E
:103A5000EEF08043903459539003B900028038E867
:103A60002402FFE0B4EE02802E8590F0B4DE030263
:103A70003B82B4BA03023BA5B4BF03023B1F5443CD
:103A800060231283F450030239F6740A126831E598
:103A9000F042900555D9921283BCE8FD14141478B5
:103AA00002F202388FC082C0837E0AE0700AA3DE71
:103AB000FAD0E0D0E0023A29D083D082E0FD0303BF
:103AC000543F539003F208A37E08E5F04290E05380
:103AD0009003F22DFD08A3DEF1EFF8E22323540357
:103AE0007006E82407F88016FEE2543FF21818E248
:103AF000D2E4F2E82408F8E2CEF208EEF208E5F0AB
:103B00004290E0539003A3C39D60111283F45003CD
:103B10000239F6C8CFC8E2D2E7F2EFF8023A8FA333
:103B2000E0FD0303543F44C0539003F208A37E0416
:103B3000E5F04290E0539003F22DFD08A3DEF1E59D
:103B4000F04290E02DFDE0B404004005B4070040D1
:103B5000027404FEC0E004539003F208A374FFF261
:103B600008D0E0C0E0FEE5F04290E0539003F22D73
:103B7000FD08A3DEF1D0E0FE740CC39E1268310292
:103B80003AFEC27FA3E0FD543F4480539003F20805
:103B9000A37E07E5F04290E0539003F22DFD08A3C9
:103BA000DEF1023AFEA3E0FD0303543F44C053900C
:103BB00003F208A37E04E5F04290E0539003F22D57
:103BC000FD08A3DEF1E5F04290E02DFDE0C0E053FA
:103BD0009003EFF8E223235403FC700508080880E3
:103BE0000EE2543FF21818E2D2E4F2E82405F8D0CD
:103BF000E0C0E0BC0004240580022406F208A3749F
:103C0000A0F2087E04E5F04290E0539003F22DFD0F
:103C100008A3DEF1BC0003023C2218E2CCF208EC5F
:103C2000F208D0E0C0E0FEE5F04290E0539003F2ED
:103C30002DFD08A3DEF1D0E02404023B77240553D8
:103C4000900FF214C0E008A374A0F208023B619048
:103C50000004E0601DB4011FE4F090345974EEF0EC
:103C600012839B1285979034591283B39034591262
:103C700083BCD2360237851283961283B3C20F807B
:103C8000F17801E2540F600C14203F0320E105B4E9
:103C9000040040030237855403C0E0D2D56003B46A
:103CA0000105E2A2E792D5081D302D0F9000EDE04E
:103CB00054F070077401F208E4F218D0E09000208C
:103CC00075F016A41268267E16123FD3BD00B430DC
:103CD000D503023D639000208583A0A88290004C0C
:103CE0007D16E2F008A3DDFA900059E004F09000A0
:103CF0005FE0541FFDA3E0541FFEE054E04DF09040
:103D0000005FE054E04EF090005EE020E00E900096
:103D100050E0C2E1F0900054E0C2E1F0900036853E
:103D200083A0A8829000627D16E2F008A3DDFA90DD
:103D3000006FE004F0900075E0541FFDA3E0541FF5
:103D4000FEE054E04DF0900075E054E04EF090003D
:103D500074E020E00E900066E0C2E1F090006AE0BE
:103D6000C2E1F0900032E0900010F0900048E09046
:103D70000011F090005EE0900012F0900074E0906E
:103D80000013F09000DEE4F0A3F0C029C02A75F023
:103D9000001279FB05F030F2F8D0E054F0532A0F0E
:103DA000422AD029900027E0A2E6920CC03AC03BFC
:103DB000D2D590007885823A85833B900020128B83
:103DC0001AD2D5901FA285823A85833B901EA212FB
:103DD0008B6AD03BD03A539003C211203E0630216B
:103DE0000902378530220302378575F0610243727C
:103DF0000243957801E2540F6005B40500400302C8
:103E00003785081DBD01028008BD02028003BD0385
:103E1000269002FC75F00CA4126826E2F008A3A319
:103E2000BD010FB440028003B44A0478018003E46A
:103E30008001E2F0023F0E9002F475F00CA41268CB
:103E400026E220E77FF008A31D7408F0A3E2F00843
:103E50001DA3E2540FF0302A1AE2C4540FB4080034
:103E60004011B40D00500CC0E0740212683CD0E068
:103E7000F0A3A3E0FEA3A3A3A3A3E82407F8E254BE
:103E8000F0F5F008E2C4540F45F0F0BE00030880DE
:103E90002715827408C39EF5F0E895F0F8E2540FF8
:103EA00018DE03F0800EF5F0E2540F18C445F0F070
:103EB0001582DEE9E82409F8ED9409FDBD000280D1
:103EC00018023DF57E04123FD308081D1D7E08121E
:103ED0003FD308081D1DBD00E8203F32C2D5302D5C
:103EE0000A9000EDE054F07002D2D5900300858373
:103EF000A0A88290031830D50390030C7D1830D50C
:103F0000027D24E2F008B8000205A0A3DDF5C03A66
:103F1000C03BD2D590033085823A85833B90030025
:103F2000128B1AD03BD03A75F004900308755A00F2
:103F3000E0B44003755AFF740C126831D5F0F112E9
:103F40006775302602D25F023DD67801E2081D5423
:103F500003600F30E005901DB0800A901E28800598
:103F60007801901D38EDB479004003023785FE12C8
:103F70003FD3C03AC03BD2D5901EA085823A8583FC
:103F80003B901D38128B1AD03BD03A023DD67801B7
:103F9000D2D580047801C2D5E26035081D90032295
:103FA00075F010A41268267E0830D5027E10123FEC
:103FB000D3BD00E4C03AC03BD2D590133285823ADB
:103FC00085833B900332128B1AD03BD03A023DD608
:103FD000024395E2F0A31D08B8000205A0DEF475C7
:103FE000A001303E0375A0022200010BA317452259
:103FF000E72E893A2B45CD516F5D1168B374557F1B
:10400000F78B99973BA2DDAE7FBA21C5C3D165DDA1
:1040100007E8A9F44BFFED0B8F173122D32E753A29
:104020001745B9515B5CFD689F74417FE38B8597B1
:1040300027A2C9AE6BBA0DC5AFD151DCF3E895F438
:1040400037FFD90B7B171D22BF2E613A0345A551BF
:10405000475CE9688B742D000108891111199922B8
:10406000212AA933313BB944414CC955515DD96628
:10407000616EE977717FF9888191099991A219AAF6
:10408000A1B329BBB1C439CCC1D549DDD1E659EEC4
:10409000E1F769FFF108791101198922112A993391
:1040A000213BA944314CB955415DC966516ED97760
:1040B000617FE9887190F99981A209AA91B319BB2E
:1040C000A1C429CCB1C0F0C03AC03BC03C753C0093
:1040D000539003E208701AE2701730D50508E21811
:1040E000701B30D50108D03CD03BD03AD0F008D37B
:1040F00022E420D505304759800308E21830473FB5
:10410000C3C0E018E2089401F53AE29400F53B538D
:104110003B0FC4540FF53CD0E09400C454F0453C30
:1041200004F53C75F003C3E53A33F53AE53B33F566
:104130003BD5F0F3853A82853B83E53C02425160F2
:1041400010C0E075F016302A0375F01FA4F53CD0BE
:10415000E0202A1920270B75F000753BAE753A7EDA
:10416000802275F002753B7F753ACE801720270BB1
:1041700075F000753B7F753AF8800975F001753B65
:10418000D5753A38B5F00CE2B53B0818E208B53AF7
:1041900002800540030240E2E275F00B302A03750D
:1041A000F0088470027401253CB438004002743772
:1041B000F5F0903FE7302A03904055E5F02393F562
:1041C0003BE5F0230493F53A18E2C3953AF53A0833
:1041D000E2953BF53B5027E5F0202A13B41706E59E
:1041E0003C60158019B42D10E53CB42C0B800FB445
:1041F0001F06E53C60028006D5F0B7024288C03A4F
:10420000C03BE53AC3202A0494A280029488F53A80
:10421000E53B202A04940B80029408F53BD03BD068
:104220003A400905F0E5F0B43888805CC0F0E53A22
:1042300075F00B302A0375F00FA4F58285F083E545
:104240003B75F00B302A0375F00FA42583F583D05E
:10425000E075F01030270375F038B5F000502923D1
:104260002354FCC0E0E5516009D0E0B5510050187E
:104270008002D0E0539003429030D50108D03CD06A
:104280003BD03AD0F008C32230D501080240E27991
:10429000437E03D3E79400F709DEF9539003202708
:1042A00032E5457045E544C4540FB40500503B2445
:1042B0000B232354FC4590F5F053440F7903C3E5D9
:1042C0004333F543E54433F544D9F38544838543CB
:1042D00082C322E545C454F0F545E544C4540F4576
:1042E00045B414005004242780C7D322A210C0D0A4
:1042F000C210C2D58008A210C0D0C210D2D5780199
:10430000800DA210C0D0D2107801E2A2E792D5E2CF
:10431000547F6053F5F0081DE27E0A20100820E764
:10432000027E08547FF2E5F090132A30D5039018EE
:104330002C75F00AA4126826123FD3BD00D1C03AF2
:10434000C03B90183430D503901D3685823A858362
:104350003B90133430D503901836D2D5128B1AD037
:104360003BD03AD0D09210023DD675F061A21BB37B
:1043700092F7C21B20150575A001800375A0027875
:10438000007441F208E539F2087401F208E5F0F230
:104390007D0402388F75F0E1203E063021D40237CB
:1043A000853022CE0237857801BD000575F0078083
:1043B00005E260F8F5F0539003126B12C0F0740040
:1043C000F5F0124EE7D0F030F148D2107531A890D8
:1043D00000107D08E4F0A3DDFC90001CF0A3F09039
:1043E000001F7D5BE4F0A3DDFC9000DE7D22F0A3E6
:1043F000DDFC12659C126722E49001007DFAF0A3B7
:10440000DDFC900200787E7D00F0A3DDFCD8F81280
:104410006B1230F24F30410BC24190001EE054FD50
:10442000F0D2F0C0F01284A4F5F090000EE4F0A3F6
:10443000F0900000F0D2107531A843900490000075
:104440007880E47D00F0A3DDFCD8F8126B12E590D3
:10445000240420270320E60A54FC5390034290B51D
:10446000F0DBD0F053900320F10330F035C218C2D6
:1044700034900004E4F0C3E5306001D390001EE006
:10448000540792E692E7F090345912839B90000013
:104490001283B31285979034591283B39034591212
:1044A00083BC20F10520F202800B75F0001273E44A
:1044B00005F030F2F8023DD6023DD675F000BD00A1
:1044C0000280057801E2F5F078007441F208E539E0
:1044D000F208742730F00A740D202D03302B02747B
:1044E00010F208746230F0027466F208C0F01270C4
:1044F000E4F208E5F0F208D0F030F02090C100E0DE
:10450000302D0B302C0690C000E0C4F4540FF2089C
:1045100090FB01E0204601E4F20880087D0674006B
:10452000F208DDFCC0F01245C7D0F030F0247D1059
:10453000202D03302B19E4F208F208E550540FFD4A
:10454000E550F40303A2E392E654704DF27D1302AA
:10455000388F900001E0F5F0A3E0232354FCA2186B
:1045600092E1F208E5F0F208900078E0F2A308E0AA
:10457000F208900330E0F2A308E0F208901834E06B
:10458000F2A308E0F208901332E0F2A308E0F20888
:10459000901EA0E0F2A308E0F208E4F208F208900E
:1045A0001FA2E0F2A308E0F208902BA4E0F2A30817
:1045B000E0F208901D36E0F2A308E0F2087400F281
:1045C00008F27D2A02388F901F237D087E08E03094
:1045D000E704A2E08004C36001D3E5F013F5F0A383
:1045E000A3DEEBE5F0F208DDE3227801E220E60944
:1045F000540F601914F5158016201511540FF51578
:10460000900102ED14F5177513C0129CB7802D2090
:1046100015FB1D1D8D170808900207E2F008A3DDA9
:10462000FA900101E02323235480F513A3E030E046
:1046300003431310751604D2D5129CB7023DD6E081
:10464000A31267AEDDF975040422780175A001306C
:104650003E0375A002E2540F6005B405004003025A
:10466000378514F5F0081D902FA823232582F582A5
:10467000E5833400F5837E02123FD3C029C02A129D
:1046800079FBD0E054F0532A0F422AD029BD00BC58
:10469000C03AC03BD2D5902FB885823A85833B90F3
:1046A0002FA8128B1AD03BD03A023DD67801E254A3
:1046B0000F60ACB4050050A714081D902FAA232347
:1046C0002582F582E5833400F5837E02123FD3BD57
:1046D00000DC203FBB902FAAE0902FB2F0902FAECD
:1046E000E0902FB6F080A9780175F000E2543F60A9
:1046F0006BB411005066E2A2E792D5A2E692F150A7
:1047000002D2F0C0F0901E9A75F0085006901F205B
:1047100075F002E2541FA4126826D0F0081DE208CA
:104720001DA2D592E7F030F10E547F700AA3E0305D
:10473000E70320E602E4F0BD00B230F003127BC8CC
:10474000C03AC03BD2D5901FA285823A85833B9068
:104750001EA2128B6AD03BD03A023DD60243957816
:1047600001C03B75F000081DE220E708C2F1A2E598
:1047700092D58011C2D575F003800A7407081DD543
:10478000E0FB024830E2541F60F1B4110050ECF538
:104790003B18E208600A30F1E2B4040050DDD23583
:1047A000C0F030F114901F2075F010A4F5F0E53B37
:1047B000541F25F075F002800A901E9A75F008E5E6
:1047C0003B541FA4126826D0F0081DE220F104A279
:1047D000D592E7F030F124547F7017A3E030E7035F
:1047E00020E60F7400F0C0F0E53B75F000124EE7D4
:1047F000D0F07406081DD5E0FB8035A37404081DB5
:10480000D5E0FBE2C0E0081DE2A2E25018202B1424
:10481000E53B302E0AB40500400AB409005005D02B
:10482000E0024395D3E092E7F0A3A3D0E0F0081DA7
:10483000BD0005D03B02473A0247667801E260E1DD
:10484000081D901F9875F00CA4126826E2541FF002
:10485000E2C4035407F5F0A3081DE2A2E192D55487
:10486000E045F0F0A3081D7E09123FD3E230D502E7
:1048700074FFF0081DBD00C5C03AC03BD2D5902BD7
:10488000A485823A85833B901FA4128B1AD03BD01B
:104890003A023DD6023DD6C2D57801304703023DEB
:1048A000D630D502081D1240C51D1D30D5011D4052
:1048B0002EC0905390037E0430D5027E01081DDE89
:1048C000FC7E07A3DEFD302A01A3E2D090F01D0894
:1048D000BD0003023DD630D5C2539003024BC67EC5
:1048E0000530D5027E02081DDEFC80E47801E2304E
:1048F000E726F5F0081DE2A2E6E5F092E7601990E0
:104900001F9875F00CA4126826E223541F4480F00F
:10491000081DBD00D9024878024395D2D578088099
:1049200004C2D57807D2107531147A017F00E2B441
:10493000FF09E4F208E2D2E7FFE4F27801C0D0C256
:10494000D51240C55005D0D0024987D0D08590F00F
:10495000C082C0837E04302A010EE07051A3DEFACB
:10496000C0F053900390001FE0304107B4F00040C6
:104970000274F0F5F020471E90000FE0B5F0004003
:1049800015D0F0D083D08253900375F0A13041034D
:1049900075F0B102439890000EE02401F0A3E034DA
:1049A00000F0900000E03400F0D0F085F090D0836B
:1049B000D08230D51B202A117E04124AA2087E0321
:1049C00030470808087E0180027E08124AA280242F
:1049D000302A107E04124AA274FFF0A37E03124A0A
:1049E000A280117E04124AA27E0330470408087E8A
:1049F00001124AA2204701A37E02124AA230E1021C
:104A0000D241E054E0FE539003E285F090545F4EB3
:104A1000F008A330D540202A0508080880057E0349
:104A2000124AA2539003EAF8BF00028003B40109BE
:104A30007E0C30D50F7E10800BEF135403FE7406EE
:104A400094002EFE08DD05D2B5023DD6DEF6E8FA6A
:104A5000BF001F02493D302ACA539003181818E2BC
:104A6000C0E018E20808080885F090F0A3D0E0F054
:104A700080B17901E2F30809EF20E003E2F30809CD
:104A80007E04E2F30809DEFA30D514EF0354036024
:104A90000EB40104E2F38007E2F308E27910F302B6
:104AA000493B539003E285F090F0A308DEF422C264
:104AB000D5780130D502081D1240C51D1D30D50125
:104AC0001D4047C082C0837E04302A010EE070057D
:104AD000A3DEFA801F8590F053900390000EC3E090
:104AE0009401F0A3E09400F0900000E09400F085C1
:104AF000F090D2B5D083D0827E0B302A027E0F3068
:104B000047027E087400F0A3DEFCBD0003023DD620
:104B100030D5A0539003024BC6C2D5780130D502E0
:104B2000081D1240C51D1D30D5011D4030C09053D9
:104B30009003E2D090081D7E0A302A010E30470211
:104B40007E07A3DEFD6008545FFEE054A04EF0BD7A
:104B50000003023DD630D5C55390038069081D80FF
:104B6000EE7801E2081D540F6009B40103024B8284
:104B7000024395E270FAC24190001EE054FDF01D20
:104B80008037C043C044C0457943E2F70809B946BD
:104B9000F912428FD045D044D043402585F090741F
:104BA00001F0A37E06124AA27E091DDEFD5390038A
:104BB000D24190001EE04402F0BD0003023DD680C9
:104BC000A20249877801D2D5E254E06015B42003EF
:104BD000024AB3B44003024B1DB4600302489B0277
:104BE0003DD6D210753114E2541FC39410FCB403A7
:104BF0000050ECE808B401157A017F007805E2B4B2
:104C0000FF09E4F208E2D2E7FFE4F278021240C5BD
:104C100050030249878590F0C082C0837E04302A09
:104C2000010EE07057A3DEFAC0F053900390001F0E
:104C3000E0304107B4F000400274F0F5F020472462
:104C400054F0B4F013900000E0601920F116A2F0C7
:104C500075F040500375F09090000FE0B5F0004003
:104C60000302498190000EE02401F0A3E03400F03B
:104C7000900000E03400F0D0F085F090D083D08236
:104C8000E8FB2408F87E04124AA2302A19BC000569
:104C9000E4F0A3800F7E01124AA2BC0103E4800469
:104CA000539003E2C0E0EBF8304704080880057E2B
:104CB00002124AA2539003E2081385F090F0539039
:104CC00003E20833FB85F090E092E7F0A320470170
:104CD000A3EBF0A3202A040808800A539003E208FB
:104CE000FBE208C0E07E01124AA230E102D241E0BC
:104CF00054E0FE539003E2545F4E85F090F0A30819
:104D0000302A17EB13FBD0E033C0E0EB92E785F0DD
:104D100090F0A3D0E0F0A3D0E0F0539003EAF8BF06
:104D200000028003B4010674102CFE800BEF1354B4
:104D300003FE740794002EFE08DD05D2B5023DD6B1
:104D4000DEF6E8FABF0003024BC67902E2F3080977
:104D5000E2F30809EF20E003E2F308E92409F9EFA0
:104D60000354032404FEE2F30809DEFA024C0B7834
:104D700001C2D5BD0106E2B40102D2D5780074416A
:104D8000F208E539F208740530D50104F208124D35
:104D9000A1E502126803F2740830D50104FD02385F
:104DA0008FE51B126803F208E51A126803F208E5A2
:104DB0001C126803C0F0F5F0E51EC42354E045F072
:104DC000D0F0F208E51D126803F208E51F1268032F
:104DD000F208227801E2B41800501712681AF51B85
:104DE00008E2B43C00500B12681AF51A08E2541F8E
:104DF0007003024E8212681AF51CE2C4035407F5D0
:104E00001E08E2607DB40D00507812681AF51D0886
:104E1000E212681AF51FE4BD0600400508E21268B8
:104E20001AF5029000EAE0540FB40619E49000DC91
:104E3000F0902022E493B4A602800ABD0700400B44
:104E400008E2B4AA0674AA9000DCF0C28C758C6AE1
:104E5000758A0075380AD28C7504FF1274CE1267F9
:104E6000AEC210D27BC029C02A75F0001279FB05B2
:104E7000F030F2F8D0E054F0532A0F422AD0290241
:104E80003DD61274540243957801E2B401059000B6
:104E9000148006B4020990001508E2F0023DD60223
:104EA00043957801E2F50D086030E230780820265D
:104EB00005850D56F557602275F000E412684EB571
:104EC0000D13126C3F20F005753504800375360410
:104ED0007405126CF405F030F2E1E2F5F0E50D1224
:104EE0004EE740BB023DD670028047C083C082C0FF
:104EF000E0E5F0B4FF0474C1800A20E707B478004D
:104F000040027478F5F0D0E0C0E023901F212582A4
:104F1000F582E5833400F583E5F0600920E706E0DB
:104F2000B481028003E5F0F0D0E0D082D083126B30
:104F30003B22C082C083C0F0901F2375F040E4F094
:104F4000A3A3D5F0FA7401126B3B7405126B3B748A
:104F50000D126B3BD0E0F5F0C0D0C2D530355270A9
:104F600007D2D575F0018005B4040050449000F3D9
:104F7000E58225F0F582E5833400F583E030E02713
:104F8000E4F0900201E539232325F0241FF090027C
:104F9000057405F0A374FFF0A3F0A3E4F0D3C0F010
:104FA0007406125F3DD0F030D50705F0E5F0B4048B
:104FB000BCC235E475F000D0D0D083D082C3227853
:104FC00001E275F0C0307808202605F556755700C7
:104FD000124EE7405B023DD67801E2F5F0740FBD5A
:104FE000020208E2124FEA023DD6C082C08390005E
:104FF000207D04FEA2E0E0A3500B6003124EE7E028
:105000006003124EE7E5822415F582E5833400F54E
:1050100083EE03DDDED083D082227803E2F5F090C8
:1050200001013015039002017401125BF5023DD6B7
:105030000243957801C03ABD021E753A0008E2F5B8
:10504000F018E2B2E7128BC875A001303E0375A0DC
:105050000208081D1D02511FE220E73D7043081D94
:10506000E2547F70030250FFF5F0753A10902D273F
:10507000E0B5F002D27CA3A3A3A3A3D53AF2E5F056
:10508000902BA375F003A4126826E4F0A3081DE298
:10509000F0A3E4F0081D02511F081DC403F53A8077
:1050A0009C54E0B42002807AB4405908E2F53AA258
:1050B000E7547F4007127C6992E08014C2D5127CCD
:1050C000A592E730E00530E4025481548375F00086
:1050D000C0E075A001303E0375A00278007441F273
:1050E00008E539F2087404F2087467F208E53AF248
:1050F00008D0E0F208E5F0F2D03A7D0702388FD010
:105100003A024395E2541F6024B41100501F081D59
:10511000901EA075F008A41268267E02123FD3BD2F
:105120000008D03A127BC8023DD6025058740308DA
:105130001DD5E0FB80E90243957801BD0500405094
:10514000E2603320E40E30E54708E2B2E4F218E210
:10515000145403D3081D540F400E75F005902D27ED
:10516000D27CD27E7E05800875F008902D777E086F
:10517000A41268268009081D081D7E04902D2312A4
:105180003FD3BD00028003BD01B612537E023785B6
:10519000024395E4BD000280037801E2F5F0780057
:1051A0007441F208E539F208740AF2087463F208EF
:1051B000E5F0F20830E7030252E0540F60030252B8
:1051C0009930F53E908000E0F4F20890C200E023B0
:1051D000A2E792E1A2E692E25407F208901F237D33
:1051E000021245CC9020157D03E493540FC4F5F0D2
:1051F000A3E493540F45F0F208A3A3DDECE4F2021C
:1052000052947D01C0F0C03AC03BED1271CFF5F071
:10521000E53A13F53AA2F0E53B13F53BA2F1E53B85
:1052200013F53B0DBD050D08080808E53BF21818FD
:10523000181880D6BD0911E53AF20808080808E5F3
:105240003BF21818181880C2BD0D0F08080808088E
:10525000E53BF2181818181880B0BD11ADE53AF208
:10526000080808080808E53BF21818181818D03B79
:10527000D03A901F237D021245CCD0F030F41508AF
:10528000080808901F437D061245CC78027410F27E
:105290007D1380027D0D02388FB40400504BFD90C9
:1052A0000200E53923232D241FF0900205740AF033
:1052B000A3E5F0C45403F0D37406125F3D402A7591
:1052C000A001303E0375A00290022EE030E00618E7
:1052D000E2D2E7F208A37D08E0F2A308DDFA80B489
:1052E000540F24BF90020180C00243957801E2541C
:1052F0001F6035B420005030081D902D8675F011C8
:10530000A41268267E11123FD3BD00E2C03AC03B12
:10531000D2D5902FA685823A85833B902D97128B0C
:105320001AD03BD03A023DD60243957801E260F8AC
:10533000081D302D14C0E09000EDE054F07008E23C
:1053400054E0B44002E4F2D0E0901F9875F00CA451
:105350001268267E0C123FD3BD00D2024878203E50
:105360000620210312537EBD000580FE7801E2B4C1
:1053700004F880F602378541FF016198FD047E073D
:10538000905377759840126583126B12E493F599E8
:105390003099FDC299A3DEF4126598229001023083
:1053A0001503900202125D6440CA2015082021C432
:1053B00075A00180062022BC75A0027800902022F2
:1053C000E493F208E2B4FF05187441F20808E27DA4
:1053D00003B40A027D06EDF2087457F208E539F2CB
:1053E000087400F20D0D0D02388F7802E230E047AC
:1053F00018E2C39420F5F00303543FB53939E5F0C2
:105400005403B4030280300475F010A404F5F07F57
:1054100010E5F0126B3B05F0DFF775A001303E039D
:1054200075A002E2C03CC03BF53C753B2075F0889E
:1054300012864DD03BD03C023785024395BD08FA19
:1054400012696E78019000EEE0651CF5F0E2B5F0AF
:10545000E9A308E0651DF5F0E2B5F0DEA308E0651C
:105460001FF5F0E2B5F0D308A3E0F5F0E2B5F0CA1D
:1054700078057E04E2F4F208DEFA78059000EA7E10
:1054800004123FD31268A1023DD612696E780074EF
:1054900041F208E539F208740AF20890001EE0545F
:1054A000C0A20E92E5302D0B202C044410800A443B
:1054B000118006440B30460104F2089000EA7E0495
:1054C000E0F208A3DEFA1818A22740047E01800249
:1054D0007E02E254F04EF2080874FFF2087E04E007
:1054E000F208A3DEFA7D0D02388F7801E254C0F590
:1054F000F0605430E7051D1D1D804CE254F0F5F0BE
:10550000B440028005B45071803D75F00F202A0927
:1055100075F00B30470375F0087804E2B4110050C1
:1055200058A4FD7803E2C0E01818E2540F7803F2A3
:105530001818D0E0F2D2D51240C5403DAE9053903D
:105540000375F0000255D630F632E2F5F0B45102A0
:10555000807DB4D113BD0221080808E2F58F08E26E
:10556000F58E12654D023DD60808E2F90830F75F66
:10557000E2F70809DDFA023DD6024395E2232354FF
:10558000FCFE0820F7167014E2701108E2B40E0B4E
:1055900008E2F5F07D0290000E803B18E2F58308EA
:1055A000E2F5820830F728E2FFEE4290EFF05390E8
:1055B0000308A3E583B4800718E2F52E023DD6B4B4
:1055C0007F08E582B4FF03023DD6DDDB023DD6E273
:1055D000B4F00050A4FD7F64780378007441F208B1
:1055E000E539F20808EFF20830F61D20F006E7F280
:1055F00008098025E58FF208E58EF208E5CBF20870
:10560000E5CAF2087D018011EE4290E0539003F26A
:1056100008A3E583B480027D01DDCDE5F0B4030687
:10562000900000E0F208E8FD7802C39403F202382B
:105630008F78007441F208E539F2087407F20874B3
:1056400000F208E551030314543FF2089020157D41
:1056500003E493540FC4F5F0A3E493540F45F0F220
:1056600008A3A3DDEC75F0FD125675F208E5F0F223
:105670007D0A02388FC2AFC03AC03BC03C900000E8
:1056800020F103902000753A00753B00753C0080C6
:1056900001A3E493253AF53AE53B3400F53BE53CBC
:1056A0003400F53CE582B5F0E8126B12E58330F189
:1056B00005B41FDD8003B4FFD8853C83E53B853A04
:1056C000F0D03CD03BD03AD2AF22024395BD03FA92
:1056D0007801E2B455F408E2B4AA028003B4BBEA4C
:1056E000F52808E2B4F0E3900018E0F5F0A3E0B587
:1056F000F00CA3E0B5F0076005B407004008902067
:1057000020E493C45407900018F0A3F0A3F0020023
:105710002E0243957801E2B4AAF708E2B455F208E4
:10572000E2B450ED78007441F208E539F2087407EC
:10573000F2087401F2087400F2089000317D03E46D
:1057400093540FC4F5F0A3E493540F45F0F208A36B
:10575000A3DDEC75F0FF125675F208E5F0F27D0A54
:1057600002388FBD04028003BD062330410B78044C
:10577000E2600675F0B10243987801E230E01290E1
:105780000004E0B402005006D20EC20F80050243AE
:1057900095C20E08E21820E715300F0C1283911203
:1057A00083BCC20FB20180061283961283B39000AD
:1057B000E0EDFE123FD31284A4C03AC03BD2D59094
:1057C00000E685823A85833B9000E0128B1AD03B3D
:1057D000D03A023DD620111BE53060171263E0403D
:1057E0001278017D0490007AE0F5F0E2B5F09F08B0
:1057F000A3DDF5780590007AE2F530F0081DA37E70
:1058000003123FD3E530C36001D390001EE092E65F
:1058100092E7F0C03AC03BD2D590007E85823A85AF
:10582000833B90007A128B1AD03BD03A023DD67857
:10583000007441F208E539F208740CF20890001E79
:10584000E054C0C0E0A20E92E5302D0B202C0444A1
:1058500010800A44118006440B30460104F20812FD
:105860004DA1D0E030E610E530700C7D06E4F20882
:10587000DDFC7D0F02388F1270E4F208E5F0F208CB
:10588000127162F5F0127192C4C0E054F045F0F26A
:1058900008D0F053F00F1271BFC445F0F20890C168
:1058A00000E0202B02540F202E01E4F20890FB01AF
:1058B000E08006202B07302E03204601E4F2087D0D
:1058C0000F02388F0243957801E2BD02028003BDCA
:1058D0000304FD088005BD01067D00E2FE8029BDB0
:1058E00007E2E2145403C0E09000D82582F58274E8
:1058F00080F0D0E090008A75F016A4126826081D8A
:105900007E06123FD3023DD6C082C083C043C0444E
:10591000C045C037C03AC03B126B128D3A8E3B7502
:105920004B0A754301754400754500753700757164
:1059300000C21AD2137E0AE54BB2E0F54B12874241
:105940004032E5432401F543E5443400F544DEE705
:10595000126B1275F000126C3F7401127428126CF5
:1059600081E53BC39401F53BFEE53A9400F53A70BE
:10597000C4BE00C1754B00D03BD03AD037D045D023
:1059800044D043D083D082023DD6780290001CE2FE
:10599000F0A318E2F0023DD67801E2B40203025906
:1059A000EFB40303025A2A08E2B45A1D12537EC010
:1059B0003F125A677801E2B401030259CCB40403E0
:1059C0000259DFB405030259E7024395125A9A12AD
:1059D0005AD2125B22D03F75F003D2210243B61295
:1059E0005A9AD03F023785125AD2125B2280F312A4
:1059F000537E126AC7F4F53AF53B753C00C2D512E6
:105A00006B12126AC7F4B53B0280F4F53B653A426B
:105A10003C75F000126C3F740A127428126C81E518
:105A20003CB4FFDB125B2202378512537E90C2002A
:105A3000E054E0F53AF53B753C00126B1290C20061
:105A4000E054E0B53B0280F2F53B653A423C75F02C
:105A500000126C3F740A127428126C81E53CB4E0A9
:105A6000D9125B22023785C0D0539003126B127596
:105A70003F40900000E0F5F07455F0439040E0F5B1
:105A80002774AAF0539003E0B45503753F00439088
:105A900040E527F0539003D0D022753E00E53E53F9
:105AA00090034290125AB4E53E2404F53EB53FED12
:105AB00053900322900000126B12E53E7E80700727
:105AC0009003007E7D74037F00F004A3DFFB04DEFF
:105AD000F622125A67753E00C2D5E53E5390034246
:105AE00090125AF8400E7401126CD1E53E2404F570
:105AF0003EB53FE653900322853EF0126B129000B4
:105B0000007E80E53E70089003007E7D75F0037F87
:105B100000E0B5F00BA305F0DFF705F0DEF1C322DE
:105B2000D322125A67400C432C07E53F6008432CF0
:105B3000088003432C05126AD440057401125B4CA3
:105B40007464127428532CF0126AD422FE432D3050
:105B5000126AFE7428127428532DCF126AFE74281C
:105B6000127428DEE822024395BD01FA7801E26052
:105B7000F5B4070050F0F5F03035447E019000F4A4
:105B8000E030E031C082C083900201EEB45F028059
:105B900007E53923232E241FF0900205740BF0A390
:105BA000E5F0B40601E4F0D3C0F07406125F3DD016
:105BB000F0D083D082BE5F02800C0EA3BE04C13041
:105BC0007E047E5F80BE900018E5F0F0A3F0A3F0A5
:105BD00030150302536A20210312537E75CBFF90C8
:105BE0000018E090653F858FF020F10390654693A3
:105BF000F5CA023785C0A8C2ACC03AC0D0C082C0C6
:105C000083C0F0C03CC03DC0E0A8828583A0E270A4
:105C10000808E2187003025CEAD0E0C0E0901F239D
:105C2000753A0020E018901F43753A1020E10F905C
:105C30001F63753A2020E206901F83753A30C2D563
:105C4000E27F0813053A5039C0E0E0B48F0575F0E3
:105C5000008024B49B09E5F0D2E4B49B22800320A9
:105C6000E71DE5F0B48B028003B49B0B125CFDF0E2
:105C7000E53A126B3B8008E5F0F0D0E0D38003D02A
:105C8000E0C3A3A3DFBD20D50913F53CD2D508E2BC
:105C900080AF13F53DE5F0C2E4B48B03025CEAD0BB
:105CA000E0C0E030E00C7E01EE126B3B0EBE11F85E
:105CB00080381890020103035403FEE5392323546E
:105CC0007C2E2420F00E9000F3A3DEFDE04401F0D2
:105CD000D2359002057405F0A3E53CF0A3E53DF054
:105CE000A3E5F0F0D37406125F3DD0E0D03DD03C88
:105CF000D0F0D083D082D0D0D03AD0A822C082C0F9
:105D000083C0D0A2E492D5903212E53A142375F004
:105D100000126826E53BC3C2D194094005D2D1A345
:105D20008002E53BF5F0D3E433D5F0FC20D508F450
:105D3000F5F0E055F08005F5F0E045F0F020D514E1
:105D400030D105740112683CE0F5F0A3E025F07055
:105D500003E48002749B75F08BA2D592F4D0D0D06E
:105D600083D08222E0A3B40103025D9DB40203024A
:105D70005DABB40303025DC4B40403025DD3B40598
:105D800003025DDFB40603025DF0B40702C322B470
:105D90000A03025E20B42103025E48D322C03AE027
:105DA000F53AD2D51272E9D03AC322A3E0F5F074E5
:105DB0000112683CE0C03A753A00128BC8127BC8E9
:105DC000D03AC322A3E0F5F0740112683CE0124E11
:105DD000E7C322E0F5F0A3E0C5F0124FEAC322A327
:105DE000A3E0F5F0740212683C7401125BF5C32263
:105DF000C082C083BD060050167D10E030E7027DF2
:105E000020541F75F011902D86A4126826800590ED
:105E100001031D1D1267AE12463FD083D082C322FC
:105E2000E020E202D322A2E092D5A3E0C03EF53EFC
:105E300012A10ED03E900106301503900206F0A389
:105E4000E5F0F0A3E4F0C3228583A0A88230190214
:105E5000D322D27E1818E2F552C394BF540F902D6E
:105E60002975F005A4126826E0D2E7F00808E220C0
:105E7000E70B20E52520E34320E240C322C03CC0DD
:105E80003B85523C753B2075F08812864DD03BD047
:105E90003CE552129D6DD27CD322A2E6C03DC03CAF
:105EA000C03B753B0085523CE492E1F53D75F0083E
:105EB00012864DD03BD03CD03DC32230E33720E4A6
:105EC00034A308E2B4C103E08008A3B4C205E070C3
:105ED0000104F208E2181854F0B4F01908E552C3AE
:105EE00094BFFDE29002078583A0A8827F007B001B
:105EF000129F18D322C0A8C2AF7D0A903292E2F05E
:105F000008A3DDFAD219C3D0A822C20BD2028005A1
:105F1000755305D20BC010C013C014C015C016C0F5
:105F200017C0D0C2D3D2D4FFC20A902022E49390EB
:105F30000200F0A3745FF0A3EFF0026030C20AC069
:105F400010C013C014C015C016C017C0D0755305BB
:105F5000920BC2D3D2D45039200A0B207A0CFF9076
:105F60000202F002601DC20A80F4FF7CFF30261C92
:105F70007C02900202E0B412027C00A3E0B4FF02B3
:105F80007C00900200E5F0D2D5126360EDF802606B
:105F900067A3E0B4F009A37D05125D64026346B413
:105FA0005F11C082C083A37D05125D64D083D0825F
:105FB00040EAE0A38583A0A882900201F0A37F06B7
:105FC000E2B4060C08E2187F1330E7027F23801248
:105FD000B4800FD20AD20B080808E2FC18E2FF18BE
:105FE000800CEFF0900205E2F008A3B40624E2541E
:105FF0001F75F011902D86A41268268583A0A882B3
:10600000EFFD1D1D1D900206300A09EFFD900200F4
:1060100080027D03E2F008A3DDFA200A4A902022E4
:10602000E493900200F09002037456F0A3E539F077
:106030007C007D00900200EF2403F5F0C017E01211
:10604000640BA3D5F0F8D017EDF0A3ECF0A3740423
:10605000F0EF2406FF9002057C09E0B40A097C11E8
:10606000A3E030E2027C0C126B12200B1F9000E0C8
:10607000E0540F700620020F0263465407B4040474
:10608000D20B8008B405F1E0A2E4920B7D03207AE4
:1060900013A20B1267B3500C75F018300B0375F098
:1060A000280262B3900200EFFE200B32C083C08250
:1060B000908000E52EF02071FCD082D083C2AC121B
:1060C0006583E0F59974FF75F00AD5F0FD20990617
:1060D000D5E0F402611AC299A3DEE7026160C2ADA5
:1060E000207A02C2AC90001BE0200A0A307A092014
:1060F0002604744A8002744B75F0CCC2D5126448F1
:10610000900200E075F082D2D512644874FF75F0F9
:106110000AD5F0FD20CE10D5E0F4DD028003026048
:106120008E75F00A0262B353C83F75F000E4C2D521
:1061300012644820F7E4A3DECA307A0775F00C74C5
:106140007E801790001BE075F003B44C0375F006D9
:10615000E58F20E10375F00674E6D5E0FDD5F0F893
:10616000207A22200A1F900201E0B45F18200B055C
:106170001264B680061264C653A8CF740512742840
:10618000DD3A026346ECFE7003026346900229206A
:106190000B2D202B07202D040E90022812659875D8
:1061A000985074FF75F080209808D5F0FAD5E0F487
:1061B0008047E599C298F0A3DEE8807C02608E7586
:1061C000F084E4C2D5126448C082C0839000E1E04C
:1061D000540F2418FBD083D082126B12747A75F09E
:1061E00080309124D5F0FAD5E0F4DBED300A0AC016
:1061F00082900229D0E0B58252BD040040027D03A6
:10620000DDBA75F0090262B353C83F740075F0003F
:10621000C2D5126448F0A3307A1A202605B403A828
:106220008016DE0714144480FE809DEE30E799B49A
:1062300080968004DE928000200A12207A1190025B
:106240002AE0B539B4A3A3E0B457AE805F805D30D7
:10625000262590022AE0C017FFEDFEE8FD900229F6
:1062600074562DF8E6C2D5126360D017603EEDF883
:10627000EEFD1264C6808290022A75F000E0B4033D
:1062800007E5F0600F0261F9B41B04A3E0C2E76206
:10629000F0A380E990022AE06003026346A312A7FC
:1062A0008BF5F090020112A78BB5F0EEC2D575F018
:1062B000088004D2D5E8FDC03DC03CC03B753B2002
:1062C000753D00300A0A902F79E0F53C540F805557
:1062D000307A20302614ED30D508785628F876002C
:1062E000945624E1F53C94DE803BE824E1F53C94AF
:1062F000DE8032900205E0F53D900201E0F53C3091
:10630000D510B45F03026340B4FF028033B4BF0012
:10631000502EC39420FD0303543FB53923ED54039D
:10632000B40302801B9000F42582F582E030D5078B
:1063300020E70DD2E7800530E706C2E7F012864D70
:10634000D03BD03CD03D1264C6C27AE5D0D0D0A2BA
:10635000E5D017D016D015D014D013D010D2AC225F
:10636000C0F0C017F5F030D507E0A2E0500D800670
:10637000E0B4A0028005E5F01263BF1F1F1F1F7568
:10638000F0A07880A3E062F0A3E030D50762F0507F
:106390000866800550016662F0F0A308E830E2026A
:1063A0007880DFE530D50DE5F0500166F0A374B0DC
:1063B000500104F0E050016665F0D017D0F022786B
:1063C0008079807008770009B984FAD32254FC449C
:1063D00002F7092404F7092414F7092448F7D32203
:1063E00090007AE0F530C00CC00D7C007D0079048F
:1063F000E02CFCED3400FDA3D9F6E0B50C07A3E0DA
:10640000B50D028001D3D00DD00C22F9ECFEEDFFCA
:10641000FC7D00E96CFCFA7B00ECC4540FFCEA6CD8
:10642000FCFAC4FD54F0C333FCED540F33FDEA6CA9
:10643000FCEEFF7E00EF6DFDFBECFAECC454F0FDCA
:106440007C00EB6DFDEAFC22C0A8307802C2AFC030
:1064500090C082C083C0E0C297532EF7908000E5C1
:106460002EF0E5F075F008D296339295D297A29669
:10647000C29792E0D5F0F2F5F0D0E0C0F075F008E8
:10648000D296339295D297A296C29792E0D5F0F227
:10649000D0F0C0E0432E08908000E52EF0D0E0D090
:1064A00083D0824390FCD090D29120D50353C83F33
:1064B000D0A822203E10C205C204C22112659875E0
:1064C000985043A890221264B6202F6B202D68C2EA
:1064D00007C206C222C0E0C0F0C082C08343A8A0A9
:1064E000201C21900018E0F5F0A3E0B5F00CA3E02B
:1064F000B5F0076005B40700400C902020E493C479
:106500005407800274019065389390001BF075F079
:10651000CCD083D082C0D0C2D512644875F0067446
:10652000E6D5E0FDD5F0F875F0847400C2D51264AC
:1065300048D0D0D0F0D0E0224C4B4A4942424C885F
:10654000C4E2F1F6FB881088C4E2ECF61090001863
:10655000E0F5F0A3E0B5F00CA3E0B5F0076005B4FA
:106560000700400C902020E493C45407800274017B
:1065700090653F858FF020F10390654693F5CA75CD
:10658000CBFF22D271C083C082C0E0908000E52E94
:0C659000F0D0E0D082D08322C27180E9FC
:09AC71000221D7000221D72F2295
:10659C00C082C083C0F0532842C090539003900037
:1065AC0000E0F5F07455F0439040E0F52774AAF044
:1065BC00539003E0B4550AD227439040E527F0806E
:1065CC0002C227539003E5F0F0D090752700D22E2D
:1065DC00D22BC22DC22C908000532EF9E52EF090B8
:1065EC008200E054DCB41C17D271E52E908000F0D0
:1065FC00C277908200E054DCB45C04D22D805090C1
:10660C008000532E3FD276E52EF0908200E054DCD1
:10661C00B4501BD277C276E52E908000F0C27790F2
:10662C008200E054DCB49006D22DD22C8021C246DC
:10663C0090FB00E0C0E07405F0E0540FB4050B745F
:10664C000AF0E0540FB40A02D246D0E0540FF0D056
:10665C00F0D083D08212696EC082C083C0F0500328
:10666C0002667D9000E8E0B40107A3E0B419028053
:10667C001C1264B61264C6D265D266126AD475F066
:10668C00007402126CD1746412742880F4202C0CE7
:10669C00302D099000EAE054F0B480D59000EBE086
:1066AC00543042289000EDE054707003202D0630D9
:1066BC00E60543278074300303540C42289000EC09
:1066CC00E0C4540F9066FA9390001FF0C247B4EEEA
:1066DC0000400330279B30270DB4F404D247800AC6
:1066EC00B4F207B38004B47F01B3922A801008225D
:1066FC005011190814287FAEEEF0F1F2F3F4128465
:10670C00A490007AE0F530900027E0A2E6920CD03D
:10671C00F0D083D08222C0E0C083C0825327F053D4
:10672C002DFC126AC7F454E0B4E0047407800270C4
:10673C000ED2B4D2B530B40320B5224408801EC4A6
:10674C0003B401028008B402028003B40403432D95
:10675C00034227902021E493232323540842271239
:10676C006775D082D083D0E022C0F0C278C226C236
:10677C001C75F004900308E030E60CD278A2E1928C
:10678C0026A2E0721C921C740C126831D5F0E8D071
:10679C00F022540375F00CA4900308126826E0A2B2
:1067AC00E2220000002222C0F0200A037503FF75CC
:1067BC00F00A4004D2AC8011D2ADC0D0BD0202C2EE
:1067CC0037D0D0800BD0D04007203627D23680056A
:1067DC00203720D237C0D0E53904232323C0F075ED
:1067EC00F0FFD5F0FDD5E0F7D0F0D5F0D8D0D0D370
:1067FC00D0F022C3D0F022C0F0C0E0C4540F75F02A
:10680C000AA485E0F0D0E0540F25F0D0F022C0F0BF
:10681C0075F00A84C445F0D0F0222582F582E58318
:10682C0035F0F583222582F582E5833400F5832249
:10683C00C0D0C582C39582C582E5839400F583D010
:10684C00D022C0D020F01420F1229000202582F517
:10685C0082E5833400F583E0D0D02290003630F10D
:10686C00EC202FE9202DE690006280E1202FEC2017
:10687C002DE990004C80D6C0F0E230E603C39407BB
:10688C00540FC4F5F008E230E603C39407540F45E7
:10689C00F008D0F022126B12C082C083C0F0C090FE
:1068AC00C2AF5390039000E875F00A7E007F007829
:1068BC006DE0F62EFEEF3400FFA308D5F0F3EEF0FA
:1068CC00F6A308EFF0F6439040126A7CC295C2978B
:1068DC00D295126A71C295126A71126A71D2957F41
:1068EC0006126A71DFFB126A7C7E10786DC295C24B
:1068FC0097D295126A71C295126A71D295126A7109
:10690C007F06EE3333339295126A71DFF8C2D57F6E
:10691C0008E6339295126A71DFF820D50508D2D5B6
:10692C0080ED74FF126B127F6EDFFED5E0F6126AFB
:10693C007C3096FD0E08BE16B4C295C297D2951245
:10694C006A71C2957F08126A71DFFB432D8090C279
:10695C0000E52DF4F0D090D2B5D0F0D083D082D217
:10696C00AF22C082C083C0F0C0D053D0E77D03C03B
:10697C0090C006C007C2AF539003439040C2971219
:10698C006A7C7E10786DC295C297D295126A71D2CC
:10699C0095126A71C295126A717F06EE3333339287
:1069AC0095126A71DFF800C2D57F08126A71A2963F
:1069BC0033DFF8F620D50508D2D580ED126A7C0EAF
:1069CC0008BE16C2432D8090C200E52DF4F0539002
:1069DC0003786D7E007F00E62EFEEF3400FF08B8D2
:1069EC0077F5E6B5060A08E6B507057041BE003E28
:1069FC009000E875F00A7E007F00E02EFEEF340078
:106A0C00FFA3D5F0F58EF0E0B5F03FA38FF0E0B525
:106A1C00F0387005BE00028031D007D006D090D27D
:106A2C00B5D0D0D0F0D083D0821268A1C322786DBB
:106A3C009000E8E6F008A3B879F9D007D006D0901A
:106A4C00D2B5D0D0C380150269817401127428DDCF
:106A5C00F6D007D006D090D2B5D0D0D3D0F0D0831A
:106A6C00D082D2AF22D29775F005D5F0FDC2972215
:106A7C0090C200432D80E52DF4F0532D7FE52DF4CD
:106A8C00F02201193423713000C082C083C0D0536E
:106A9C00D0E77D009000E8C083C082906A8EED93B1
:106AAC00D082D083F0A30DBD07EDD0D0D083D0829F
:106ABC00C322126AC7F4541FF53922C082C08390D6
:106ACC008000E0D083D08222C082C083C0E090C11D
:106ADC0000E52CB2E4B2E5B2E6B2E7F0D0E0D08348
:106AEC00D08222C082C08390C200E0540FD083D0E9
:106AFC008222C082C083C0E090C200E52DF4F0D0A9
:106B0C00E0D083D08222532DBF126AFE432D401257
:106B1C006AFE22C082C083C0E0E526F490C3C03078
:106B2C002D03908200540FF0D0E0D083D0822270DD
:106B3C000122126B12302D05B4040050F4C0E0E5B4
:106B4C0031543F7003753101E532543F7003753297
:106B5C0001E533543F7003753301E534543F700342
:106B6C00753401D0E0B40500500D127162532CF055
:106B7C00422C126AD4C322B40D005011127192C06F
:106B8C0082C08390EF02F0D083D082C322B4110074
:106B9C0050111271BFC082C08390EF04F0D083D02B
:106BAC0082C322B441004002D322C082C083C0F011
:106BBC00F5F0901F21232582F582E5833400F583BF
:106BCC00E0C0E0E5F014C0E0C4145403F5F0E5397E
:106BDC002323547C25F02420900201F090020574AC
:106BEC0003F0A3D0E0540F04F0A3D0E0F0D23505AD
:106BFC00F09000F3A3D5F0FCE04401F0D37406123E
:106C0C005F3DD0F0D083D08222700122C082C0833D
:106C1C00C0E023901F212582F582E5833400F583A3
:106C2C00E030E704A2E08004C36001D3D0E0D0835D
:106C3C00D08222C0E0E527547FB46003D0E022204C
:106C4C002F06202D0320F11120F005432D20800369
:106C5C00432D10126AFED0E022C082C083908000C7
:106C6C0020F005532EEF8003532EDFE52EF0D0835A
:106C7C00D082D0E022C082C083C0E0202F06202D1D
:106C8C000320F11420F005532DDF8003532DEF90DA
:106C9C00C200E52DF4F0801190800020F005432E09
:106CAC00108003432E20E52EF0D0E0D083D082223A
:106CBC0020F009753500C25BC25D80B9753600C223
:106CCC005CC25E80B0C03AF53A126C3F7408127424
:106CDC0028126C817408127428D53AEDD03A22200F
:106CEC00E003026C81026C3F801D20F00CD26470BA
:106CFC0002C264C265F531800AD2677002C267C2F3
:106D0C0066F532126AD42230F1E020F00CD23070E9
:106D1C0002C230C231F533800AD2327002C232C2A2
:106D2C0033F534126B1F22702520F11120F006C2AE
:106D3C0064D2658004C267D266126AD42220F0063F
:106D4C00C230D2318004C232D233126B1F22800A7D
:106D5C00D2E74003F53122F53222540F601BA2F02A
:106D6C00202FED202DEA202B033046E430F1E1D228
:106D7C00E74003F53322F5342220461A202B172046
:106D8C00F009C264D2657531058007C267D2667599
:106D9C003205126AD42230F1E620F009C230D23129
:106DAC007533058007C232D233753405126B1F223E
:106DBC0020F10D20F004C2658002C266126AD42252
:106DCC0020F004C2318002C233126B1F22C0F0C00B
:106DDC0082C0838525F0740B12684E30E21974055D
:106DEC00126CF4126C3F20F007753502C25B800503
:106DFC00753602C25C80178525F07460126D337491
:106E0C000712684E20E30280057402126CD1D08305
:106E1C00D082D0F022C0F0126EB5C0E0901E9CE57E
:106E2C003B75F008A4126826E0A2E7D0E0C0E0921F
:106E3C00E7F0A3A3E0F5F0C0F075F000740212685F
:106E4C004E543FB53B11126CBCC0F0E5F0540375C9
:106E5C00F014127961D0F005F0202D0530F2DD80B0
:106E6C000330F1D8127C1DD0F0403915F0740712A4
:106E7C00684E30E12F20E42CD0E0B4440040027482
:106E8C00440303543FC0F075F00FA4D0F020F00A77
:106E9C00F535D25BA2F1925D800CF536D25CA2F195
:106EAC00925E8002D0E0D0F022740C12684E543FF7
:106EBC00127BCEE5824004940280029405F582E5B3
:106ECC00839400F583C0F0E0540F75F005A404D052
:106EDC00F022C090C082C083539003C0F08525F08F
:106EEC00741212684EF5F0E52554039000102582BB
:106EFC00F582E5833400F583C2D5201308E06008E1
:106F0C00147004D2D5E5F0F0D0F0D083D082D090BC
:106F1C00228525F0801475F000800F75F001800A31
:106F2C0075F002800575F0038000C0F0126C3F74A0
:106F3C000712684E20F00D75350230E303753505E8
:106F4C00C25B800B75360230E303753605C25CC03C
:106F5C003B740212684E543F6025F53BC0F075F04F
:106F6C0008901E9EA4126826D0F0E5F0540304F09D
:106F7C00E53B1271CF50087432127428126E21D076
:106F8C003B7405126CF4740C12684E127BCE7405B3
:106F9C0012684E4004A3A3A3A3E0547F70030270B5
:106FAC0040C03AC0E0A3E0540FC0F075F005A40453
:106FBC00D0F0F53A740012684ED0F07802C082C05E
:106FCC0083E0543F605CC0E0901F21232582F58252
:106FDC00E5833400F583E054C0B4C004D0E08042B3
:106FEC00E5F0B47A02800DE0B48302801930E71624
:106FFC00D0E0802EE0700474838021B4830474008C
:10700C00801AD0E0801CE5F0B4780040027478B4AB
:10701C00010AE538C394057401500104F0D0E01264
:10702C006B3BD083D082A3E030E603853AF018B8EE
:10703C00008BD03AD0F0228525F0740112684E54A2
:10704C003F601EC0E0901F21232582F582E583342A
:10705C0000F583E030E703D0E022E4F0D0E0126BDF
:10706C003B22C03AC03FC0F0F53A753F0305F074BF
:10707C001512684E541FB53A0A740012684E126C01
:10708C0015400FD53FE7E53AD0F0D03FD03A12711A
:10709C00CF22D0F0D03FD03A22E550540F20641AC2
:1070AC00206717203014203211302D08908200E018
:1070BC005403800690C3C0E0540FC0F0F5F090C2AA
:1070CC0000E054E0302C04C2E58005302D02B2E61D
:1070DC0045F0D0F022126B12C082C083302D0C759B
:1070EC00F00090C000E0540F02715D302F2990C267
:1070FC0000E003A2B3B392E3A292B392E4A2B2B3C0
:10710C0092E5A2B4B392E6547F304202541F30434E
:10711C000254E7F5F08036302E1430421130430E15
:10712C00204603E4800490FB03E0F5F0801FA2B33B
:10713C0092E0A29292E1A2B292E2A2B492E3F4544F
:10714C000F3042025403304302540CF5F090C0004F
:10715C00E0D083D08222C082C083C03AC0F0901F9E
:10716C0023753A04E030E704A2E08004C36001D345
:10717C00E5F013F5F0A3A3D53AEAC4540FD0F0D040
:10718C003AD083D08222C082C083C03AC0F0901F14
:10719C002B753A08E030E704A2E08004C36001D309
:1071AC00E5F013F5F0A3A3D53AEAD0F0D03AD083AA
:1071BC00D08222C082C083C03AC0F0901F3B753A87
:1071CC000480A1C03A8F3AC03BC0F0C082C083C3D8
:1071DC00F53B6008B4110040187400C3400630F64B
:1071EC0003D3B2E0D083D082D0F0D03BAF3AD03AC8
:1071FC002275F00090001DE0B53B02D2F6E53BC0D5
:10720C00F075F008901E9AA4126826D0F0E0A2E760
:10721C0092F2302E06A3E0A2E792F3E53BB4050010
:10722C004008B409005049302B22302E1F30F31C7B
:10723C00AF3B90C100302C0890C000E0C4F4800734
:10724C0030F70390FB01E013DFFD92F190C00030AA
:10725C00F70390FB03AF3BE013DFFD92F092E230BB
:10726C00F103D3800465F0A2E2E5F054030271E867
:10727C00C3E53B9408F53B202F39302E0C204605F6
:10728C00E4C30271E8D2F780A4B401082043CCA275
:10729C00B3B380C7B402082043C1A292B380BCB47C
:1072AC0003082042B6A2B2B380B1C32042ADA2B44F
:1072BC00B380A890C200E003A2B3B392E3A292B34E
:1072CC0092E4A2B2B392E5A2B4B392E6547F3042F8
:1072DC0002541F30430254E7AF3B027264E53A702C
:1072EC000122C0F0C082C083901F9875F00CE53A63
:1072FC00A4126826E054E07007E53A12736A8057CE
:10730C0030D554B4E002804FC082C083C03B753B83
:10731C002075F00C12864DD03BD083D082A3A3A352
:10732C00A3A3A3E07006C3125F3D802BB4FE1075BF
:10733C00F005A3E060031273ADA3D5F0F68018B48A
:10734C00FF15E5255403042582F582E5833400F509
:10735C0083E060031273ADD083D082D0F022901FF3
:10736C00A275F00CA4126826E020D506B47E3180FC
:10737C0001E4B47E06748BA2D592E4B47A02748FC5
:10738C00B47F027487F5F0C03B740A12683CE0F5D8
:10739C003BA3A37401125BF5A3A32330E4F7D03B0A
:1073AC0022C082C083C0F0F53A901F9875F00CA4EF
:1073BC00126826E054E0700CE53A12736AD0F0D0F3
:1073CC0083D08222B4E002808EA3A3A3A3A3A3E064
:1073DC007004C3125F3D80E5C0F0C083C082900092
:1073EC00D8E5F054032582F582E5833400F583E477
:1073FC00F0E5F0540375F016A4900080126826E4B2
:10740C00F0A374FFF0A3F0A3E4F0A375F01274FFE3
:10741C00F0A3D5F0FBD082D083D0F022C0F0F5F0F1
:10742C00C0A275A200C083C08290DDBAE58F30E1A6
:10743C000390EEE3A3E58370FB126B12D5F0EAD058
:10744C0082D083D0A2D0F022C0A8C0E0C2AFC0D0FE
:10745C00C09053D0E7D29600C297D31274A4C00741
:10746C0074BF1274C2D296C000C00678197E077F12
:10747C0008C297A29613D297DFF7F608DEF18519AA
:10748C0002D006D000D007C297C31274A4D090D2F9
:10749C00B5D0D0D0E0D0A822C083C082908000E5C7
:1074AC002E92E0F52E800990C100E52C92E3F52C8C
:1074BC00F0D082D083227F08C297139296D297DFA6
:1074CC00F722C0A8C2AFC0D053D0E7C090D296006C
:1074DC00C297D31274A4C007748E1274C2740012B3
:1074EC0074C2D007C297C31274A4D296C297D31297
:1074FC0074A4C00774BE1274C2D296850219C0005F
:10750C00C00678197E07E61274C208DEF9D006D0E0
:10751C000074801274C2D007C297C31274A4D090A6
:10752C00D2B5D0D0D0A822758C6A758A00D28CB214
:10753C000D300D05B22020200132C0F0C0E0C0D0CB
:10754C00C082C083C09053900343D018B212301243
:10755C00030276A690001CE0600714F07003A3E40D
:10756C00F0E531543F6026B40111C264C265C2100B
:10757C0075310075F00012793A800FE53114F53150
:10758C0030E602B26430E702B265126AD4E53254D6
:10759C003F6024B4010FC267C26675320075F001FA
:1075AC0012793A800FE53214F53230E602B26730C8
:1075BC00E702B266126AD4E533543F6027B4011275
:1075CC00C230C231753300202D4775F00212793A62
:1075DC00800FE53314F53330E602B23030E702B2F7
:1075EC0031126B1FE534543F6027B40112C232C212
:1075FC0033753400202D1A75F00312793A800FE59B
:10760C003414F53430E602B23230E702B233126B86
:10761C001FE535603F14F535205B0BA2E7547F70F6
:10762C00187535008015702CC25B7535F8A25D920B
:10763C00E175F00F127961801B501975F000A25D95
:10764C0092F1126CEBE535B4FD027535FF7005B2A5
:10765C00F1126C81E536604214F536C3205C0BA246
:10766C00E7547F701A7536008017702EC25C753621
:10767C00F87401A25E92E175F00F127961801B50D3
:10768C001975F001A25E92F1126CEBE536B4FD02B5
:10769C007536FF7005B2F1126C81D27D201226E591
:1076AC000314F5037015E54AB4AA03128E25E503FD
:1076BC00D236D237200204D202D25A541F7006128C
:1076CC00654D1264B61538E538600DD090D083D076
:1076DC0082D0D0D0E0D0F0327910901E9CE975F0B9
:1076EC0008A4126826E0A2E7547F60041492E7F025
:1076FC00D9E8E553600B14F5537006755305126405
:10770C00C6902BA67901E06003B4FF030277B5B4F1
:10771C00FE030277C154C0B4C00BE0543F600314A5
:10772C0044C0F0800FE502B4597FE014B401047436
:10773C00FCD27CF07073A3A3E020E107E4F075F0B9
:10774C0000805CA2E092E7C2E1F04050307E1EC0A7
:10775C0082C083902D2775F010E0A3A3B51904E027
:10776C00D2E3F0A3A3A3D5F0F0D083D08230262CA3
:10777C00C082C08375F000741012684EB51914E500
:10778C00F0C0F075F008902D77A4126826D0F0E0C8
:10779C00D2E3F005F030F2DFD083D08275F0FE74C6
:1077AC000212683CE5F0F0D27CA3A3A309B98002D5
:1077BC00801F027712E502B401EFA3E0127BF6A35F
:1077CC00E0F5F092E665F030E6E1E4F075F000806B
:1077DC00CEE50220E02F20E102D2589000DEE054EA
:1077EC001F600EE014F0541F7007F0532C9F126AA8
:1077FC00D4A3E0541F600EE014F0541F7007F05334
:10780C0026F5126B1F75F000900080E030E72FA278
:10781C00E6541F604914701F1273E4307840C0F0B6
:10782C00C0255325FCE5F05403422575F01412A62F
:10783C0027D025D0F0802792E6D2E7F08020601E7A
:10784C00B40102801914F0B4011474082582F58275
:10785C00E5833400F583E04401F0740E8002741665
:10786C0005F020F20C2582F582E5833400F5838047
:10787C009A7901901F23E020E70A600814F0700445
:10788C00E9126B3BA3A309203505B911E98003B9B3
:10789C0041E4300E1A900004E06014900003E060A4
:1078AC000E14F0700AD2169000E2E0900003F0750E
:1078BC00380AE5022401D4B46001E4F502541F70C7
:1078CC0003127454E50260028053D214D259307EF4
:1078DC0002D27BE554600215542042062043031269
:1078EC0089D1C029C02A75F0001279FB05F030F25D
:1078FC00F8D0E054F0532A0F422AD029902FBA79AD
:10790C00C8A3A3E0600214F0A3D9F6EA700FD27BEF
:10791C007904900014E0600214F0A3D9F853D0E776
:10792C00BCFF030276D71CBC00F97CFF80F5C03A83
:10793C00E412684EF53A901F2123126831E054810D
:10794C00B48006E4126D33800964817005744012B2
:10795C006CF4D03A22C082C083C0255325FC42254A
:10796C00900308C0F075F00CA4126826D0F0E0303B
:10797C00E10312A627D025D083D0822232C082C048
:10798C0083E5F054032323902FA82582F582E58309
:10799C003400F583E0A2E520F11520F009900014E5
:1079AC00E090002C801C900015E090004280132089
:1079BC00F009900016E09000588007900017E090B6
:1079CC00006E5003C380067004E0127BCEE582404B
:1079DC0004940480029407F582E5839400F583E017
:1079EC00C0E0A3A3A3E0A2E7D0E0D083D0822274AE
:1079FC000212684EA2E79257127989F5299254C067
:107A0C0082C0839000E0E0A2E0920EC03AE41268DB
:107A1C004EF53AC0F053F003E5F0600E15F0E412A9
:107A2C00684EB53AF3D0F0027AEFD0F0753A00E533
:107A3C00F054032323902FA82582F582E58334008C
:107A4C00F583E030E005753A80802030E105753A29
:107A5C0081801830E407C24FC24E027AEF304F05D6
:107A6C00753A808006304E03753A81740012684E68
:107A7C00C2F7C082C083543F605CC0E023901F21DA
:107A8C002582F582E5833400F583E0B4832CC08233
:107A9C00C083740C12684E543F127BCEE5824004B6
:107AAC00940380029406F582E5839400F583E0D07C
:107ABC0083D082B47A028002801454C0B4C004D043
:107ACC00E08013E53A7007E030E70620E103E53A81
:107ADC00F0D0E0126B3BD083D08220F706D2F7A314
:107AEC00E0808F300205305402C24A53F003753ADD
:107AFC0009C0F005F0E52A13153AD5F0FA92F0A278
:107B0C004A13D53AFCF52AA2F0D0F0D03A126B12F7
:107B1C00304A574055C090C03AC03BC043C044C0E7
:107B2C0045C03F90000085833A85823B75430175C3
:107B3C004400754500539003439004753F04740A48
:107B4C00302A010430470274072582F58250020561
:107B5C0083E04440F01282CA50E4D03FD045D04478
:107B6C00D043D03BD03AD090D2B530F14A901F22BE
:107B7C00C0F0C02175F001E0A2E7547F6024500AE8
:107B8C00C0F0127C69B3D0F08003127BF6A3E03016
:107B9C00E70320E60EE450027481F0E5F0126B3B33
:107BAC008001A3A305F0E5F0203505B411C98003CD
:107BBC00B441C4D021D0F0D083D08222C082C08303
:107BCC0080ABC082C0837003C3801AB48000501590
:107BDC0090132AC0F0C0E075F00AA4126826127C3B
:107BEC00A7D0E0D0F0D083D08222C082C083C36003
:107BFC001BB480005016C0E0C0F090182C75F00A31
:107C0C00A4126826E0D0F0127CA7D0E0D083D082FA
:107C1C0022901E9AE53B75F008A4126826C083C01A
:107C2C0082E0547FB47F03D38022E5822406F58260
:107C3C00E5833400F583E0127C69F5F0A3E0C0F035
:107C4C00127C69D0F045F030E607A2E0D082D083F8
:107C5C0022D082D083E0547F127BF6B3227004745E
:107C6C0080D322B4800050F7C082C08375F003909B
:107C7C002BA3A4126826E0F5F0A3600BA3E0235419
:107C8C0001A2E04440800DE0547F127BF670027438
:107C9C00805480B3D083D08222D322755B00127DB6
:107CAC0003C0F04009E51E54077003C3803DC0D0EB
:107CBC00C083C082142582F582E5833400F583E00D
:107CCC00D082D083D0D05005B47F0280D8C3601B43
:107CDC0090032275F010A412682675F004127D73BF
:107CEC005009127D735003D5F0F3B3D0F0E55B145B
:107CFC0030E203755B0522C083C082C0F075F0B41E
:107D0C00901D38C0F0E0035430F5F0E0541F1268B9
:107D1C001A651C543F7046A3E0540F12681AB51D27
:107D2C003DE0C4540F45F06013245EB46404740049
:107D3C0080044002946412681AB51F22D0E075F0DA
:107D4C0008B43D004009B47900400674088004056D
:107D5C00F005F0D3E5F0D0F0D082D08322A3A3D0ED
:107D6C00F0D5F09FC380EFC0F0C0E0E0A3541FF546
:107D7C00F0E51B126803B5F002800E5003C38001BE
:107D8C00D3A3D0E0D0F0055B22E0543FF5F0E51A28
:107D9C00126803B5F00280E850E6C380E475370042
:107DAC00757200C213E525540390008375F016A478
:107DBC002582F582E0540375F00CA4900300126840
:107DCC0026E0A2E792D5A3E00430D50424060303F1
:107DDC0003540FB4040050027404FEA3A3E0043057
:107DEC00D5042406030303540FFDC2D5A3A3A3A3F8
:107DFC00C082C08390008AE525540375F016A41246
:107E0C0068267871E0F608A3B877F9E0F549A3E0A5
:107E1C00F54A8525F0740B12684E30E208D083D0F9
:107E2C00827537012230191D902D29E552C394BF5C
:107E3C0075F005A4126826E054037004A21D92E0AC
:107E4C005329FC4229D083D08220482E204907E5B3
:107E5C0049B4FF028024D2D5E549700AE54A700680
:107E6C007537030281337871E4F608B875FBA649BF
:107E7C0008A64A8EF07E02027ED9ED60FAA8823006
:107E8C004C0478077D0485833FE525540375F01673
:107E9C00A49000891268267F04C000C005C082E04F
:107EAC001582F5F0853FA0E2B5F00B18DDF1D0821C
:107EBC00D005D0008014D082D005D000304C06E81C
:107ECC00240CF8DFD44337408003204C0D12813C46
:107EDC00E53792E0F53730E00722753701027FA5D0
:107EEC00853A83853B82E53F429030D54AAEF075AA
:107EFC006D00756E00786DBE06028005BE0401082B
:107F0C0008E0F608A3B873F9BE06087408126831C5
:107F1C00E0F572E525540375F01690008AA41268FA
:107F2C0026539003786DE6F0A308B873F9853A836D
:107F3C00853B82E53F4290304729C082C08375F073
:107F4C0004E0701BA3D5F0F9D083D082D3539003F7
:107F5C00757300757400757500757600027EDCD043
:107F6C0083D082A3A3E05477F5F0A3E05477A33039
:107F7C002A01A3786D30470EC5F0F608A6F008E08C
:107F8C00A3F608760008E0F608A3B877F953900337
:107F9C00201A4C201949304C06D2135337BF2220DB
:107FAC002A19202806E56F547F8028E56FA2E7E5A3
:107FBC0071030392E6547F60EC80183029E420288A
:107FCC0004E57480F0E574A2E7E575030392E654CA
:107FDC007F60D87006753780028133127BCEB3E593
:107FEC003792E3F537304946E56DB49907E56EB441
:107FFC009902803AE549B56D0BE56EB54A064549DF
:10800C006024802AE56E2401D492F0B54A18E56DFF
:10801C00A2F03400D4B5490E7007E54AB4010280D1
:10802C0005433704800843370280030280F5201A89
:10803C00FA2019F7304A37E57220E2EF8525F07403
:10804C001312684EE0541FF5F0A3E0541FB5F0175F
:10805C007015A229B392E7A228B392E5657354A0D8
:10806C00700C4337108007E573541FB5F0F4E52509
:10807C0054032323902FAA2582F582E5833400F53F
:10808C0083E0F5F0E572A2E492E1A2E692E25407F5
:10809C00B5F0005003433708E57220E24C8525F01B
:1080AC00740C12684E127BCEE5824004940280025E
:1080BC009405F582E5839400F583E0C4540F6029A0
:1080CC00E525540375F096A4902FBA12682675F026
:1080DC0032E0B5430EA3E0B5440AA3E0600B43378E
:1080EC00108006A3A3A3D5F0E8302A158525F074DB
:1080FC000712684E30E00AE576543FB40103D38092
:10810C0020E57230E508127D035003433708E57112
:10811C00302A05302902E575202804A2E08002A24D
:10812C00E1E53792E5F537E53754FB7002D21322BF
:10813C00204703028249C0F030D5030281E490004D
:10814C0003539003439004753F04300C18A88285A8
:10815C0083A08583F07F047976C3E2977035181974
:10816C00DFF80281F7A8828583F07F047976C3C299
:10817C00AC85F0A0E2D2AC9770071819DFF1028140
:10818C00F7740CC39F28F8B403E005F0E5F0B48055
:10819C00D98013740CC39F28F8B403B905F085F08B
:1081AC00A0E5F0B480AF126B12300C02C2ACE53F0C
:1081BC0053900324046021F53F4290300C0375A0CA
:1081CC000075F000E5516007B53F02800B400930A7
:1081DC000C03028161028176126B12D3753A007521
:1081EC003B00900000539003D0F02208888285F069
:1081FC008385833A85823B75F003853A44853B43FE
:10820C00C3E54413F544E54313F543D5F0F2E543D8
:10821C002401F543E5443400F5F0540FF544E53FF3
:10822C000303543F20F40114C0E0C454F04244D082
:10823C00E0C4540FF545126B12C3D0F022900050DD
:10824C00E493B4550AA3E493B4AA0412005222C0D6
:10825C00F08EF0BE060215F07477C39EFD90000000
:10826C00539003439004753F0475450085833A850C
:10827C00823B754301754400C3AFF0EDF830D51067
:10828C007404302A01042582F582E5833400F583D9
:10829C00E096701FA308DFF8BE0611E5822409F5ED
:1082AC0082E5833400F583C3E0967007C3126B122A
:1082BC00D0F0221282CA50C1126B12D0F022304779
:1082CC002EA3E583B4801E126B12E53F539003245A
:1082DC00046014F53F4290900000E5516007B53FF3
:1082EC000280044002C322D390000053900322E585
:1082FC00432401F543E5443400F544500205452080
:10830C002A16E53B240BF53BE53A3400F53AB47FED
:10831C0044E53BB4F63F8014E53B240FF53BE53ACE
:10832C003400F53AB47F2EE53BB4F829126B12E514
:10833C003F53900324046025202705B44002801D80
:10834C00F53F4290753A00753B00E5516007B53F2B
:10835C0002800A4008853B82853A83C322D3753A52
:10836C0000753B0090000053900322900005539041
:10837C0003E0C0E0A3E0C0E0A3E0F582D083D0E04E
:10838C0054FC42902290000880E490000B80DFC0E7
:10839C0082C083900005E59054FC539003F0A3D069
:1083AC00E0F0A3D0E0F022C082C08390000880E609
:1083BC00C082C08390000B80DDC09053900390006E
:1083CC0005E0F5F0900008E0B5F019A3E0F5F090A9
:1083DC000006E0B5F00EA3E0F5F090000AE0B5F071
:1083EC0003D09022D3D09022C082C083C0905390EF
:1083FC000390001EE030E308C3D090D083D08222DB
:10840C00D2E3F0D090D083D08212841D128391D30A
:10841C002290001E539003E030E4141283777414FE
:10842C0012683112845F400D60051284C58006907D
:10843C0034595390031283B31283911283BC22E5F7
:10844C0082B4590DE583B43408E59054FCB40001B2
:10845C0022D322E583B47F028004500B8038E5825E
:10846C00B4EE005002802FE59054FC6013202707D7
:10847C00B43C004007E422B4F80050F97401C32264
:10848C00C082C0831284A4D083D082B4400330272E
:10849C00E470E9C380DFD322C0905390039000E3D3
:1084AC00E0543F70053027087437304102743A04A9
:1084BC00543F2323F551D09022E59054FC53900364
:1084CC00600824044290900000221284A4429090F0
:1084DC000000223018047404D322128377E0B4EE27
:1084EC000122903459539003E0B4EE012254F0B4BD
:1084FC00B00474148002740A12683112845F40E86C
:10850C0060051284C580E1D3539003740322128456
:10851C005F400D601874FFF0A3E58270F81284C5FB
:10852C0012839B12837712859753900322C090532A
:10853C009003C082C083C0F075F004900024E0204A
:10854C00E5147404126831E020E50B7412126831E2
:10855C00D5F0EBC38001D3D0F0D083D082D0905033
:10856C001674EEF012839BD21853900390001EE009
:10857C00D2E5F0D374042253900390001EE0D2E4B1
:10858C00F090345912839B12859722C0F0C0D01200
:10859C008377C082C083C2D51283C54026128391D3
:1085AC00E0B4EE02801D54F0B4B004741480027474
:1085BC000AC0E01268311283B31283911283BCD0CB
:1085CC00F0800375F00A12837774EEF0A3D5F0FBFC
:1085DC0020D507D2D512839B80BED083D082128344
:1085EC009B128377D0D0D0F022C0F0E51B12680329
:1085FC00F5F0E054E045F0F02DFDA3E51A12680308
:10860C00F5F0E54520E701E453457F030354C045ED
:10861C00F0F02DFDA3E502126803C0E0235460F5D1
:10862C00F0E51C12680345F0F02DFDA3E51D126862
:10863C0003F5F0D0E0C454F045F0F02DFDA3D0F0DC
:10864C00229000E0E0540BB4086390020174FFF038
:10865C00900205E53B6006B4201620F2507409F038
:10866C0090020AE5F0F0A3E53CF0A3E53DF08010A4
:10867C007408F090020AE53BF0A3E5F0F0A3E4F0F7
:10868C009000EEE0900206F09000EFE0900207F010
:10869C009000F0E0900208F09000F1E0900209F0F8
:1086AC00D3C0F0740A125F3DD0F0400122C2ACC0BE
:1086BC00F01284DFD0F05003D2AC2274DEF0A3E5CC
:1086CC003B44C0F0FDA3E4F053457F1285F5E53B38
:1086DC0020E510701FE53CF02DFDA3E53D2DFDE5DB
:1086EC003D801430F2EF74FFF02DFDA3E53A2DFD23
:1086FC00E53A8003E4F0A3F0A3E5F0F02DA3F0A39A
:10870C0012851A900004E0046001F0300E25B401CB
:10871C000DD2169000E1E020E706B2018005C216EA
:10872C009000E2E0C0E0900003E06004D0E0800341
:10873C00D0E0F0D2AC221284DF500122C2ACC2D500
:10874C00201A06201903126EDE8537F030190BE55E
:10875C0052C394BF540F44208005E52554030423D1
:10876C002330F00D20F10AD2E0C0E074BFF0A3D0AA
:10877C00E0F0FDA3E43013027420A2F292E6A2D53D
:10878C0092E730F00720F104A2F692E6F020F00315
:10879C004345801285F530F05F30F1055337F18099
:1087AC0057C083C082C090539003E525540375F0E5
:1087BC000CA4900300126826E0A2E7A3E004500486
:1087CC002406030303540FB4040050027404D09025
:1087DC00D082D083F0F5F0FF2DFDA37477C39FF802
:1087EC00E6F02DFD08A3DFF8740CC395F0FFE4F060
:1087FC00A3DFFCEDF0A3802BE54BF02DFDA3E543AF
:10880C00F02DFDA3E544F02DFDA3301A04E53E80C8
:10881C0009E5378571F0A2F092E2F0C0D02DD0D0EE
:10882C00A3F0A3E53730130292E0A2D592E7F53717
:10883C0012851A900004E0046001F0300E25B4019A
:10884C000DD2169000E1E020E706B2018005C216B9
:10885C009000E2E0C0E0900003E06004D0E0800310
:10886C00D0E0F030137FE57120E07AC03CC03DE5EC
:10887C0025540375F096A4902FBA1268267F327592
:10888C00F0FFA3A3E0540F6017C395F05009E0F577
:10889C00F085823C85833DA3DFE8853C82853D8362
:1088AC00C3E5829402F582E5839400F583E543F0F9
:1088BC00A3E544F0A3C082C0838525F0740C126834
:1088CC004E543F127BCEE582400494028002940504
:1088DC00F582E5839400F583E0C4540FD083D082F5
:1088EC00F0D03DD03CC3D2AC221284DF500122C266
:1088FC00ACC2D5201A06201903126EDE74BAF0A38E
:10890C00E5255403042323A2F092E0F0FDA3E43008
:10891C0013027420A2F292E6A2D592E7F0434580AE
:10892C001285F5C083C082C090539003E525540393
:10893C0075F00C900300A4126826E0A2E7A3E004F3
:10894C0050042406030303540FB4040050027404AF
:10895C00D090D082D083F0C0E02DFDA3E54BF02D5C
:10896C00FDA3E543F02DFDA3E544F02DFDA3E53774
:10897C00F02DFDA3D0E0FFC0A8C2AFC082C083C061
:10898C0090539003E525540375F016A490009012B3
:10899C006826C3E5829FF88583A0D090D083D082CF
:1089AC008FF0C090539003E2D090F02DFDA308DF20
:1089BC00F17408C395F0FFE4F0A3DFFCEDF0A3D055
:1089CC00A802883C22C03D753D008005C03D753D28
:1089DC0080539003C03CC082C083C03AC03B753CFE
:1089EC0000C2D590007885823A85833B9000201296
:1089FC008B1A5017433C0175F000E412684E540F6B
:108A0C00F0A3E0540FF005F030F2EFC2D590033034
:108A1C0085823A85833B900300128B1A5003433CAA
:108A2C0002C2D590183485823A85833B9013341258
:108A3C008B1A5003433C04C2D590133285823A857D
:108A4C00833B900332128B1A5003433C08C2D590DF
:108A5C001EA085823A85833B901D38128B1A5003D9
:108A6C00433C10C2D5901FA285823A85833B901E51
:108A7C00A2128B6A500F433C40901F42753A60E43F
:108A8C00F0A3D53AFBC2D5902BA485823A85833BC3
:108A9C00901FA4128B1A5003433C80C2D5901D36F4
:108AAC0085823A85833B901836128B1A5003433DCE
:108ABC0001C2D5902FB885823A85833B902FA8129E
:108ACC008B1A5003433D04C2D59000E685823A854B
:108ADC00833B9000E0128B1A5003433D08E53D2088
:108AEC00E7117004E53C600BD27F753B0075F0100C
:108AFC0012864DD03BD03A900001E53CF5F0F0A346
:108B0C00E53D547FF0D083D082D03CD03D22C03D97
:108B1C00C03E753D00753E00126B12E0253DF53DE3
:108B2C00E53E3400F53EA3E582B53AEFE583B53B6F
:108B3C00EA30D509E53DF0A3E53EF08009E0B53D0E
:108B4C0008A3E0B53E03C38001D3D03ED03DC08323
:108B5C00C082900001E4F0A3F0D082D08322C03D0B
:108B6C00C03E753D00753E00126B12C0F075F010E2
:108B7C00E0253DF53DE53E3400F53EA3E05480256F
:108B8C003DF53DE53E3400F53EA3A3E0253DF53D26
:108B9C00E53E3400F53EA3A3A3A3A3D5F0D2901FCA
:108BAC002275F040E0253DF53DE53E3400F53EA351
:108BBC00A3D5F0F0901FA2D0F0028B3DC0D0C082A4
:108BCC00C083C0F0C03AC03BA2E792D5547FB480BA
:108BDC00004003028CB0F53BC2407005D240753B9F
:108BEC007FC03BC03A533A83C0F0C0D0C03C307E0B
:108BFC002C753C10902D27E0B53B1AD27C20D5402B
:108C0C00E5F0B4FE10A3E0B4010274FCF5F0D2D58B
:108C1C00753A82802B7405126831D53CDA753C04A8
:108C2C00900030E0B53B11D27C20D514E5F0B4FEB9
:108C3C0007740112683C80CE7416126831D53CE37F
:108C4C00D03CE53B85F03B75F003902BA3A4126858
:108C5C002675F000E0D2E0B4FF02D2F1E53BF0D291
:108C6C00E0B4FF02D2F0E53A30E70375F001A3E07F
:108C7C00547F6002C2F1127BF6A3E030F10723446B
:108C8C00025403F53A30F002543C533A03453A92FD
:108C9C00E6A2D592E7F0D0D0D0F0D03AD03B30401D
:108CAC0003D53B0DD03BD03AD0F0D083D082D0D07E
:108CBC0022028BED74FF22201A0330190122C0D03E
:108CCC008525F030D509740712684EA2E092D57450
:108CDC001412684E541FC0A853A8EDC0E075A00133
:108CEC0078FFE545F218E544F218E543F2C0D0D21E
:108CFC00D51240C55007D0D0D0E0028DA7D0D0748B
:108D0C000A302A010430470274072582F582E58374
:108D1C003400F583D0E0C0E07003E0541FA229B307
:108D2C0092E7A228B392E5F030D511302A0EA3A316
:108D3C00A3E0543F6006146003E014F0539003D09A
:108D4C00F0E5F060569000E0E030E54FA2E4920BC5
:108D5C00D0A8740A127428C0A853A8EDC2D5E54552
:108D6C006002D2D5900203742230D5067426F0A38B
:108D7C007445F0A3E543F0A3E544F0A330D504E536
:108D8C0045F0A3E5F0F0740430D5027406200B0511
:108D9C00125F0A8006202D03125F10D0A8D0D022BB
:10A7950020202020454E5452414E43452F20202055
:10A7A50020454E5452414E43452F20202020454EF2
:10A7B500545245452F20202020454E5452414E43AA
:10A7C500452F2020202020455849542F2020202087
:10A7D50020455849542F2020202020534F525449BA
:10A7E500452F2020202020455849542F2054524ED3
:10A7F5002E20434F44453D2F2054524E2E20434F8B
:10A8050044453D2F20434F44452054524E2E3D2F65
:10A815002054524E2E20434F44453D2F414C41522A
:10A825004D205A4F4E45204E6F2E2F414C41524DD3
:10A83500205A4F4E45204E6F2E2F5A4F4E452041E0
:10A845004C41524D45204E2E2F414C41524D205AE0
:10A855004F4E45204E6F2E2F414C4C20414C4152BE
:10A865004D205A4F4E4553202F414C4C20414C41D1
:10A87500524D205A4F4E4553202F544F5554455352
:10A88500204C4553205A4F4E45532F414C4C2041A7
:10A895004C41524D205A4F4E4553202F205245468C
:10A8A5004C455820204E6265722E2F205245464C4D
:10A8B500455820204E6265722E2F205245464C4544
:10A8C5005845204E756D722E2F205245464C4558E1
:10A8D50020204E4265722E2F20204A4F4220434FA2
:10A8E5004445204E6F2E2F20204A4F4220434F448F
:10A8F50045204E6F2E2F2020434F4445204A4F427E
:10A90500204E6F2E2F20204A4F4220434F44452092
:10A915004E6F2E2F202D2D3E2041524D4544202097
:10A92500202020202F202D2D3E2041524D45442012
:10A9350020202020202F202D2D3E2041524D454501
:10A945002020202020202F202D2D3E2041524D4516
:10A95500442020202020202F202D2D3E2044495307
:10A9650041524D45442020202F202D2D3E20444985
:10A975005341524D45442020202F202D2D3E20446B
:10A98500455341524D45452020202F202D2D3E2059
:10A9950044495341524D45442020202F2121212156
:10A9A5002041524D45442021212121202F212121C3
:10A9B500212041524D45442021212121202F2121B3
:10A9C50021212041524D45452021212121202F21A2
:10A9D5002121212041524D45442021212121202F93
:10A9E5005354415455533A20502E41524D4544201D
:10A9F5002F5354415455533A20502E41524D4544FE
:10AA0500202F5354415455543A20502E41524D4510
:10AA150020202F5354415455533A20502E41524D26
:10AA25004544202F2D2D2D2044495341524D454459
:10AA3500202D2D2D2F2D2D2D2044495341524D458F
:10AA450044202D2D2D2F2D2D2D2044455341524D84
:10AA55004545202D2D2D2F2D2D2D20444953415277
:10AA65004D4544202D2D2D2F202D2D3E2052454383
:10AA75004F524445442020202F202D2D3E20524565
:10AA8500434F524445442020202F202D2D3E204564
:10AA95004E5245474953545245202F202D2D3E20D7
:10AAA5005245434F524445442020202F20434F44D4
:10AAB500452052454A454354454420202F20434FC5
:10AAC50044452052454A454354454420202F2020E3
:10AAD500434F44452052454A4554452020202F20C8
:10AAE500434F44452052454A454354454420202F71
:10AAF50020202041435449564154454420202020DC
:10AB05002F202020414354495641544544202020BC
:10AB1500202F202020204143544956452020202025
:10AB250020202F202020414354495641544544209C
:10AB35002020202F20204E4F542052454C45564171
:10AB45004E5420202F20204E4F542052454C455620
:10AB5500414E5420202F4E4F4E205349474E4946D3
:10AB65004943415449462F20204E4F542052454CCD
:10AB75004556414E5420202F20496E6E206F6E2081
:10AB8500616C61726D2120202F20496E6E206F6EE1
:10AB950020616C61726D2120202F20496E6E206529
:10ABA5006E20616C61726D6520202F20496E6E20CC
:10ABB5006F6E20616C61726D2120202F2020202076
:10ABC500436F6E74696E7565202E2E2E2F20202002
:10ABD50020436F6E74696E7565202E2E2E2F2020F2
:10ABE500202041726D656D656E74202E2E2E2F20EE
:10ABF500202020436F6E74696E7565202E2E2E2FD2
:10AC0500434F4D4D414E442041424F5254454420FF
:10AC15002F434F4D4D414E442041424F52544544E0
:10AC2500202F434F4D4D414E444520414E4E554CEE
:10AC350045452F434F4D4D414E442041424F5254BF
:10AC45004544202F2043415244204E6F2E2F204350
:10AC5500415244204E6F2E2F4241444745204E6FAE
:0CAC65002E2F2043415244204E6F2E2F12
:108DAC00C0D0A2B5D208302F15C0E07405D5E0FDB7
:108DBC00D0E030B309D0D032C0D0A2B4C2089224D3
:108DCC00C082C083C0E090C200E0A2E4B39209D09C
:108DDC00E0D083D082C0E0C0F0C082C083E52754CD
:108DEC000F75F003A4908DF573028E92029214020B
:108DFC0092140291450299EF029A4802911E028E3A
:108E0C00920291EF02911E02911E02911E02911E7E
:108E1C0002911E02911E0291EF12659C126722C0F4
:108E2C00D0C2AFC21FD288D28AA24292A8A24392C9
:108E3C00AA126B12C289C28BD0D0D2AF2222C03000
:108E4C00D031C832D833C134D135C936D937C2380C
:108E5C00D239CA43DA0A19300031013202330834EC
:108E6C0009350A3610371138123918431A0AF030FE
:108E7C00E131D232C333B434A535963687377838DE
:108E8C0069395A434B0AC2A8C2AAC2AFC0905390C8
:108E9C000353D0E7C000C001C005C0079032CA859B
:108EAC0082787F2DA22492F0C224D31298CB7E0814
:108EBC00C31298CB4037A2D5C0E0E5F033F5F0D023
:108ECC00E0A2D5202410500574FF99800AD224907A
:108EDC0032CA7F2D7E0833C0E0D31298CBD0E0305D
:108EEC002402DECCF0A3DFC6D2AF02912B126B12A0
:108EFC0030240633DEFDF08076E578240BB58256FF
:108F0C009032B37F08E4C0E0A3E0B4B9028001B3AF
:108F1C00D0E033DFF1F5F09032B3E0908E4AB4B983
:108F2C0005908E62800240F97F0CE493B5F03AA371
:108F3C00E4934480C0E09000D8E5215403F5F0257B
:108F4C0082F582D0E0F0126C3F740A127428126C15
:108F5C008174101274284388055388F5A24292A894
:108F6C00A24392AAD2AF029114A3A3DFBD80E7E57E
:108F7C0078B5820CE5F0F4F5F0908E7A7F0C80AA2F
:108F8C00C0A09032A28583A0A8829032CA7E08C26B
:108F9C0024C2D5D225E47F062038027F04C0E0E548
:108FAC00782428B58205D0E0029019E033F0DE0376
:108FBC00A37E08D0E0B35002B2251320241220382F
:108FCC0005B458D98003B48AD4D22475770080C3F1
:108FDC00DFCBC0E0E033F0DE03A37E08D0E0500529
:108FEC003025058028302525203802030303036231
:108FFC007720D52075A032F208B8000205A02038E1
:10900C0005B40F078003B41F02D2D58086D0A0D23E
:10901C00AF02912B20380563770B8003637705E54E
:10902C007770EAE8B5782A7800E2B40C04744380CF
:10903C0009B40D04740A80024430D0A04480C0E00E
:10904C009000D8E52154032582F582D0E0F0028F00
:10905C0062E578241EC3984010600EFFE475A032C0
:10906C00F208B8000205A0DFF7D0A0C0A0C2D5E579
:10907C0021540375F00CA490030030D50390030227
:10908C00126826E0FFA3E030D50B6066B408004000
:10909C00027408800470027408CF9032A28583A0F9
:1090AC0025822F14F820D508EF30E0040F08E4F2E5
:1090BC00E521540375F016A490008F30D503900071
:1090CC0089126826C0827E0630D5027E04E4F01533
:1090DC0082DEFBD082E2540FDF03F08015FE18E233
:1090EC00540FC44EF0158218DFEB20D505D2D502F3
:1090FC00907BE52154039000D82582F582E58334DA
:10910C0000F5837480F0D0A0D007D005D001D0003A
:10911C00D090D083D082D0F0D0E0D0D0D2AF3285F6
:10912C0021F053F0037444126D337F0AC31298CBB1
:10913C004002DFF8128E2880CFC2A8C2AAC2AFC0EC
:10914C009053900353D0E7C000C001C005C00790F6
:10915C0032A27F20A22440418011D31298CB50021E
:10916C008064C31298CB40FA20D52E7E08D224D32B
:10917C001298CBC31298CB5002804BA2D55002B29E
:10918C0024E013F0DEE9D31298CBC31298CB20D590
:10919C000520240580052024028084D31298CBC39B
:1091AC001298CB30D5F3B43B02801BB42400401290
:1091BC00B42E00500DC39423B40A01E4F0A3DF9A3B
:1091CC008004740F80F6BF200302912BBF00028035
:1091DC0005E4F0A3DFFC7F0AC31298CB4002DFF852
:1091EC0002907702911E32D21DC0D0C0E0C0F0C0F8
:1091FC0082C083C09053900353D0E7C000C001C01D
:10920C0005C007C0060292ECC21DC2A8C2AA300C4F
:10921C0002C2ACC09053900353D0E7C000C001C051
:10922C0005C007C006C0A8C2AF78777E087F41E4AE
:10923C00D31298CB402CC31298CB402B30D509D3EA
:10924C001298CB401DC38007D31298CB4014D33354
:10925C001FBF0005D0A80292DDDEDBF608E47E0815
:10926C0080D4D0A80298B1D0A80EB878005062B8BB
:10927C0077F2BF3E028007BF3AEA540F8005A22462
:10928C00B392E3B40F0050DC4430B43A047443801E
:10929C0013B43B04740A800CB43C0474438005B4CE
:1092AC003E02740AC0905390034480C0E09000D8F2
:1092BC00E52154032582F582D0E0F0D09043900252
:1092CC004388055388F5A24292A8A24392AA029819
:1092DC0089DE03F68005C33380F7F67442C39FFD25
:1092EC00740112994CA224B3E57792E7F577E52146
:1092FC005403F55CC224E55C540375F016A490008D
:10930C002B126826E020E60302939FE55C5403755C
:10931C00F00CA4900300126826784CE0F6A308B871
:10932C0050F9E54C30E711E5822405F582E0701E1A
:10933C00E54D547F24028016B4110CBD2303029317
:10934C00F5BD304C0293F590945604232393B50548
:10935C00030294232404B50537E521540375F01654
:10936C00A4900083126826E5772354F0440CF07522
:10937C004F00C224E54C30E714534C7F20390812BF
:10938C00990350030298B153770702943202944028
:10939C0002940BE55C540375F00CA4900300126866
:1093AC0026784CE0F6A308B850F9E54C30E711D21A
:1093BC00D5A3A3A3A3A3E020243BD22460598035DA
:1093CC002024146052B42002804A20394A201D47C0
:1093DC00F9C2D5D2248007B501028002D2D5B411CE
:1093EC000DBD23028003BD3016C2240296859094D5
:1093FC005604232393B50502801DB4FF0280180583
:10940C005C535C03E5215403B55C0630D509029826
:10941C00B102930202977AC224E54C30E716203948
:10942C0005129903401CE54C30E706534C7F5377EB
:10943C007F029780E54D7003754D08E54CB41A001A
:10944C0040030298B12323909457730294BFFF02F8
:10945C0094D41A0294E62C0295081A02950C1A025E
:10946C00951BFF029523240295412502955E30023F
:10947C00957422029583250295BA2002960E40021D
:10948C00961D2002962F20029665200296703002BF
:10949C009685FF02973D2C029655220294BFFF023F
:1094AC00956C40029751220297572502975D160240
:1094BC009763FF754C81E54D2323F54D04F54EE57F
:1094CC004F2323F54F02942A754D90754C01754F1F
:1094DC0088754E1102942A0298B1203903BD2CF7DD
:1094EC0020390A537CF0740612995B70EA754C04AF
:1094FC00754D28754E00754F00029780D22480C898
:10950C00754D98754C01754E00754F0002942A7577
:10951C004DA8754C8180EF203903BD24BA20390A3F
:10952C00537BF0740512995B70AD754C04754D202E
:10953C0080C10298B1203903BD25F720390C79255B
:10954C007E087877E612993640E8754D24754C0103
:10955C0080A1203903BD30DA754D30754C0080F098
:10956C00203903BD40CC80F0754D18754C01754FFA
:10957C0000754E0002942A203908BD25B5129903B6
:10958C0040B053777F740412994CED2404FDC077DE
:10959C00C078857977857A78D07AD079754D94753D
:1095AC004C01754F90754E190297800298B1203975
:1095BC0003BD20F7740212994C0D0D53773F2039DF
:1095CC0035E5775438B428E3C2D5C22578777E04C4
:1095DC007F11E630D50133335002B22533DF0F2033
:1095EC00D5072025C6D2D580E13025BF8008DEE71F
:1095FC0008E67E0480DD537707754D9B754C02029F
:10960C0094FF203903BD40A3754D18754C0002948E
:10961C00FF203903BD2094754DA0754C00754F008B
:10962C000297807448C39D12994CC07CC07D857F85
:10963C007C857E7DD07ED07F754D20754C00754F1E
:10964C0000754E00C2D50297A0203906201D03BD1F
:10965C002204744980CF0298B1203903BD20F775DC
:10966C004D2080B6203903BD30EC754D90754C0003
:10967C00754F90754E10029780BD2304C2D580059E
:10968C00BD3054D2D530390302971E7F2230D5021B
:10969C007F2F78777E07E6339225335002B225DF91
:1096AC000520250A8031DEF208E67E0880EC7F1664
:1096BC0030D5027F1E7877E6333392257E0630D57F
:1096CC0003337E057903D905337903800D335002BA
:1096DC00B225DF0630250B0298B1DEEA08E67E08DB
:1096EC0080E47F1730D5027F1F7877E6337E0779C9
:1096FC000330D503337E06D905337903800C335000
:10970C0002B225DF0520250A80CDDEEB08E67E08B7
:10971C0080E553773F754C0120D50B754D94754FF3
:10972C008C754E15804E754D96754F97754E1880ED
:10973C0043203903BD2CA0754DA8754C04754F0002
:10974C00754E12802F754D20029577754D20029520
:10975C0077754D90029577754D38754F00754E00A5
:10976C00C374409D12994CEDF57FC2D58026434EB3
:10977C008002961D78779032A2E6F0A308B880F9A3
:10978C00C2D5854CF030D503854EF0C374489D2569
:10979C00F012994CE54D30D502E54F547FFF790816
:1097AC00787FE4D333DF02800AD9F856F6187908AB
:1097BC00E480F056F6E418F6B8780050F9C071C0A1
:1097CC0072C073E54D30D502E54F20E704787F80F9
:1097DC00101299A57873E54EB41206756E00756F6C
:1097EC0000E54E30E706756F00757000E5215403F7
:1097FC0075F016A490008F7F0630D5059000897FF8
:10980C0004126826E6F0181582DFF920D51BD073F8
:10981C00D072D071E54F603578779032A2E0F6A324
:10982C0008B880F9D2D502978E30241BE582240724
:10983C00F582E572C4FFE573C4540F4FF0A3E573D2
:10984C00C454F0FFE04FF0D073D072D071E52154C6
:10985C00039000D82582F582E5833400F58374806B
:10986C00F0E521540375F016A49000832582F5824F
:10987C00E5833400F583E0535C03455CF0D006D0FF
:10988C0007D005D001D000D090439002D083D08275
:10989C00D0F0D0E0D0D0D2ACC289C28BD2A8D2AAA0
:1098AC00301D0122327F0AC31298CB4002DFF885AB
:1098BC0021F053F0037444126D33128E2880BE795C
:1098CC00FF7D2420080C400530B21A801120B215FF
:1098DC00800C400530B316800520B311800000DDEC
:1098EC00E2D9DED3227D02DDFEA2B480067D02DD4C
:1098FC00FEA2B592D5C322C3301D0122ED14141360
:10990C0092D53400FFF90978777E07E63392253338
:10991C005002B225DF0530250AD322DEF208E67E9E
:10992C000880ECC22530D5108001335002B225D905
:10993C0007202502D322C322DEF0087E08E680EA47
:10994C00FF78777E09C3E613F608DEFADFF322FF11
:10995C00E478776608DFFCFFC46F540F2206871982
:10996C00476736004294967296000268435456003C
:10997C00001677721600000104857600000006556B
:10998C003600000000409600000000025600000067
:10999C00000016000000000001786D760008B87415
:1099AC00FA797B9099687F02E7C4540F6018FEC364
:1099BC0078737406C0E09336D4F618D0E0D5E0F492
:1099CC00E63400F6DEE9DF02800EA3A3A3A3A3A373
:1099DC00E7540F6003FE80D7A3A3A3A3A3A309B9E5
:1099EC0080C422D2B2D2B3C2A8C2AAC090539003F0
:1099FC0053D0E7126B12E521540375F00CA49003BD
:109A0C0008126826E030E721547FB43002801AF542
:109A1C00F0E527548045F0F527D090439002D08391
:109A2C00D082D0F0D0E0028DE1D090439002D08370
:109A3C00D082D0F0D0E0D0D0128E2832D2B2D2B3B5
:109A4C00C2A8C2AA126B12C2AFC09053900353D0DB
:109A5C00E7C000C001C005C0077E07787776000814
:109A6C00DEFB78777F08D37964129B614010C37951
:109A7C0064129B614008D37934129B61500D029B98
:109A8C0048C37934129B6150ED8021743499B4022F
:109A9C000040EBB406004005B4070040E1B3E633E8
:109AAC00F6DFDE7F0808B87FD8029B487877790606
:109ABC00E46608D9FC70C7E57753770F54E0B420FF
:109ACC0006C208C2098019B46006D208C209801007
:109ADC00B44006C208D2098007B48060D208D2090B
:109AEC0085797F85787E85777D757C00757B00C058
:109AFC0071C072C0731299A5E5215403C0E075F0D2
:109B0C0016A490008C12682678707F04E6F008A3E7
:109B1C00DFFAD0E0D073D072D0719000D82582F5E6
:109B2C0082E5833400F5837480F0D2AFD007D00582
:109B3C00D001D000D09043900202911ED2AFC20847
:109B4C0074641274288521F053F0037444126D333D
:109B5C00128E2880D77D10E58F30E1027D08200819
:109B6C000C400530B21B801120B216800C40053021
:109B7C00B30F800520B30A80000000DDE1D9D6D3F5
:049B8C0022C322329C
:00000001FF
